:100000000C9407040C942F040C942F040C942F04CC
:100010000C942F040C942F040C9405370C942F048B
:100020000C942F040C942F040C942F040C942F0484
:100030000C942F040C942F040C94BD380C946E393E
:100040000C942F040C942F040C942F040C942F0464
:100050000C9496360C942F040C942F040C942F04BB
:100060000C94BB360C9426380C9450370C942A37D9
:100070000C942F040C944C360C942F040C942F04E5
:100080000C942F040C942F040C94E0360C947136CD
:100090000C94C2370C949C370C9476370C942F0434
:1000A00007634236B79BD8A71A39685618AEBAAB61
:1000B000558C1D3CB7CC5763BD6DEDFD753EF617F5
:1000C0007231BF000000803F08000000BE9224494A
:1000D000123EABAAAA2ABECDCCCC4C3E000000807A
:1000E000BEABAAAAAA3E00000000BF000000803FED
:1000F0000000000000084178D3BB4387D1133D19AD
:100100000E3CC3BD4282AD2B3E68EC8276BED98FD9
:10011000E1A93E4C80EFFFBE01C4FF7F3F0000001D
:100120000000010008191304E81A0010191302E86E
:100130004C0011191301E8820010191301E8B400F2
:1001400011191301E8EA0010191302E81C01101933
:100150001302E84E0111191301E8000303070F3FD2
:10016000FFFF07070707070707070707070707072F
:100170000707070707E01FF83FFC7C3E700FF00FF2
:10018000E007E00700070007000F001E003C00F832
:1001900003F007C01F003C00380070006000E00062
:1001A000FFFFFFFFFFFF07F007FE07FF8783C38006
:1001B000F38039C01CE00E0007000F007F003F00F5
:1001C0001FE00078001E00070003F001F800FE00A9
:1001D000770073E0F8FFF83FF807F00000380038C8
:1001E000007800F800F801F803B8033807380E3833
:1001F0001C381838383870386038E038FFFFFFFF97
:10020000FFFF0038003800380038003800381FFF82
:100210000FFF8FFFC700038001C000E000700039AE
:10022000F03FFE1FFF8F83E700F0003C000E000749
:1002300000038001C000FC00EF0073C0F0FFF83F36
:10024000F807E00003E00FF81FFC3C1E380E700EAC
:1002500070006000E000E3E0EFF8FFFCFC3EF00E11
:10026000F00FE007E007E0076007700F700E3C3EFC
:100270003FFC1FF807E0FFFFFFFFFFFF0006000E37
:10028000001C001800380070006000E000C001C0D1
:100290000180038003800700070007000E000E00A6
:1002A0000E000C001C001C0007F00FFE0FFF8783E0
:1002B000C780F38039C01CE00E780F1E0F07FF01C6
:1002C000FF03FFE3E0F9C01DC00FE003F001F800F9
:1002D000FC00F70073E0F8FFF83FF807F000005A61
:1002E000012201310038003800000000003E5B4F61
:1002F0005B3E3E6B4F6B3E1C3E7C3E1C183C7E3C86
:10030000181C577D571C1C5E7F5E1C00183C180093
:10031000FFE7C3E7FF0018241800FFE7DBE7FF3023
:10032000483A060E2629792926407F050507407F91
:1003300005253F5A3CE73C5A7F3E1C1C08081C1C04
:100340003E7F14227F22145F5F005F5F06097F01FA
:100350007F006689956A606060606094A2FFA294E5
:1003600008047E040810207E201008082A1C0808B3
:100370001C2A08081E101010100C1E0C1E0C303801
:100380003E3830060E3E0E06000000000000005F02
:1003900000000007000700147F147F14242A7F2A1E
:1003A00012231308646236495620500008070300E0
:1003B000001C2241000041221C002A1C7F1C2A082C
:1003C000083E08080080703000080808080800008F
:1003D00060600020100804023E5149453E00427F03
:1003E000400072494949462141494D331814127F52
:1003F0001027454545393C4A4949314121110907F2
:100400003649494936464949291E00001400000072
:100410004034000000081422411414141414004144
:1004200022140802015909063E415D594E7C121101
:10043000127C7F494949363E414141227F41414139
:100440003E7F494949417F090909013E41415173B4
:100450007F0808087F00417F41002040413F017F25
:10046000081422417F404040407F021C027F7F04ED
:1004700008107F3E4141413E7F090909063E415136
:10048000215E7F09192946264949493203017F0126
:10049000033F4040403F1F2040201F3F4038403F27
:1004A000631408146303047804036159494D43003D
:1004B0007F4141410204081020004141417F040274
:1004C000010204404040404000030708002054540B
:1004D00078407F28444438384444442838444428E9
:1004E0007F385454541800087E090218A4A49C783C
:1004F0007F0804047800447D40002040403D007F98
:100500001028440000417F40007C047804787C0877
:100510000404783844444438FC182424181824244B
:1005200018FC7C08040408485454542404043F4430
:10053000243C4040207C1C2040201C3C4030403C5F
:1005400044281028444C9090907C4464544C4400BF
:100550000836410000007700000041360800020123
:100560000204023C2623263C1EA1A161123A40400F
:10057000207A38545455592155557941225454788C
:1005800042215554784020545579400C1E52721225
:1005900039555555593954545459395554545800AE
:1005A00000457C410002457D420001457C407D12B2
:1005B00011127DF0282528F07C5455450020545414
:1005C0007C547C0A097F4932494949323A444444BF
:1005D0003A324A4848303A4141217A3A42402078FA
:1005E000009DA0A07D3D4242423D3D4040403D3CFB
:1005F00024FF2424487E4943662B2FFC2F2BFF0920
:1006000029F620C0887E0903205454794100004413
:100610007D413048484A32384040227A007A0A0AFE
:10062000727D0D19317D2629292F28262929292671
:1006300030484D4020380808080808080808382FB6
:1006400010C8ACBA2F102834FA00007B0000081440
:100650002A142222142A14085500550055AA55AA16
:1006600055AAFF55FF55FF000000FF00101010FFB6
:1006700000141414FF001010FF00FF1010F010F011
:10068000141414FC001414F700FF0000FF00FF1402
:1006900014F404FC141417101F10101F101F14144E
:1006A000141F00101010F0000000001F1010101098
:1006B0001F10101010F010000000FF10101010108C
:1006C00010101010FF10000000FF140000FF00FFCA
:1006D00000001F10170000FC04F414141710171466
:1006E00014F404F40000FF00F71414141414141488
:1006F000F700F7141414171410101F101F141414FB
:10070000F4141010F010F000001F101F0000001F64
:1007100014000000FC140000F010F01010FF10FF97
:10072000141414FF141010101F00000000F010FF2C
:10073000FFFFFFFFF0F0F0F0F0FFFFFF0000000010
:1007400000FFFF0F0F0F0F0F3844443844FC4A4A94
:100750004A347E02020606027E027E026355494149
:10076000633844443C04407E201E2006027E020280
:1007700099A5E7A5991C2A492A1C4C7201724C3094
:100780004A4D4D303048784830BC625A463D3E496B
:100790004949007E0101017E2A2A2A2A2A44445F0F
:1007A000444440514A444040444A51400000FF0103
:1007B00003E080FF000008086B6B08361236243611
:1007C000060F090F06000018180000001010003076
:1007D00040FF0101001F01011E00191D1712003CFE
:1007E0003C3C3C00000000000901809611800A3A60
:1007F00081550A3601082A04000000F02B0400008D
:10080000014021800A13800A29800A002E3A11240F
:100810001FBECFEFCDBFDFE3DEBF18E2A0E0B8E23E
:10082000E3E1F1EB02C005900D92A637B107D9F7CD
:100830002EE2A6E7B8E201C01D92AB30B207E1F7A5
:1008400014E0C7E0D4E004C02197FE010E946A557D
:10085000C630D107C9F70E94BD3B0C94D2560C9408
:10086000000090E0FC01E855F141E081EF3F39F1F3
:10087000845C9041DC012C91822F880F880F880FB7
:100880008E0F8033E0F490E0880F991FDC01A75BA6
:10089000B44D6D937C938751954DDC011D921C9254
:1008A000B0E22B9FC00111249C5F4096E80FF92F06
:1008B000F11D8081887F808380818160808308959D
:1008C000CF93DF93EC0189819A81DC01ED91FC915A
:1008D0000280F381E02D41E050E00995019761F439
:1008E00089819A81DC01ED91FC91008CF18DE02DE4
:1008F00061E0099591E0811190E0892FDF91CF911E
:100900000895FC0154894589252F30E0842F90E01B
:10091000821B930B541710F0CF96089501970895FA
:10092000FC0192898389981761F0A389AE0FBF2FCC
:10093000B11D59968C9193899F5F9F73938B90E023
:1009400008958FEF9FEF0895FC019289838998178E
:1009500031F08389E80FF11D818D90E008958FEFCC
:100960009FEF0895FC0192892389892F90E0805C94
:100970009F4F821B91098F7399270895CF93DF931F
:10098000EC01E881F9810680F781E02D0995EC857D
:10099000FD8586818F738683EC85FD8585818F75C6
:1009A00085838B898A8B198ADF91CF910895CF93A4
:1009B000DF93FC0194898589C485D585981306C089
:1009C0008D818F7D8D83DF91CF910895A589AE0FA5
:1009D000BF2FB11DA75ABF4F2C91858990E001967A
:1009E0008F739927858B80E48C83A485B5851296B7
:1009F0002C93948985899813E6CFA485B58515969F
:100A00008C9115978F7D15968C9387898823D9F2C1
:100A1000808D80931301178AD6CFDC011C96ED914F
:100A2000FC910FB607FE03C0258125FD04C024817B
:100A300025FD0C94D7040895EF92FF920F931F9316
:100A4000CF93DF93EC0181E0898B9C898D8998138A
:100A50001CC0AC85BD8514968C91149785FF15C07C
:100A600012966C93AC85BD8580E414968C93EC85CE
:100A7000FD8585818F7D858381E090E0DF91CF9139
:100A80001F910F91FF90EF9008958091110180FFC9
:100A900008C080911301888F8E898093130181E0B3
:100AA0008F8BF62E0C8910E00F5F1F4F0F731127ED
:100AB000E02E8D898E1104C0CE010E940D05F9CF64
:100AC000EC89EC0FFD2FF11DE75AFF4FF0820C8BE4
:100AD000EC85FD8585818062CECFCF93DF93FC01CD
:100AE00021892223C9F0EC018091110180FF08C007
:100AF00080911301808F86898093130181E0878B19
:100B0000EC85FD85858185FD03C0848186FD04C05B
:100B1000CE010E940D05F4CFDF91CF910895AF92E1
:100B2000BF92CF92DF92EF92FF920F931F93CF93DA
:100B3000DF936C017B018B01040F151FEB015E013C
:100B4000AE18BF08C017D10759F06991D601ED91D1
:100B5000FC910190F081E02DC6010995892B79F770
:100B6000C501DF91CF911F910F91FF90EF90DF9022
:100B7000CF90BF90AF900895EF92FF920F931F9385
:100B8000CF93DF93C82FD0E0A09695E0CC0FDD1F68
:100B90009A95E1F7E984F82EFF0CFF0CFF0C01E0B9
:100BA00010E08E2D8023A9F02F2D210F30E0220F91
:100BB000331FF901E75BF44D80819181892B49F066
:100BC0000190F081E02D2751354DD9018D919C91F7
:100BD00009951F5F000F183021F7E986DF91CF914B
:100BE0001F910F91FF90EF900895FC01A485B585AA
:100BF00011968C91119781FD1BC06C9182898F5F3A
:100C00008F739389981739F0A289AE0FBF2FB11D4A
:100C100059966C93828BE756FF4F808191810097A4
:100C200041F0DC01ED91FC910190F081E02D0994FF
:100C30008C91089581E00895CF93DF9390E0FC01BB
:100C4000EE5DF04120812F3F89F06330710570F433
:100C5000FC01E45CF041A08130E2A39FD0011124AB
:100C6000BC5F6130710529F411962C93DF91CF910F
:100C7000089588559141EC01E881EF3F89F0CD015D
:100C80004096E80FF92FF11D9FB7F89412962C9318
:100C900080816230710539F4886080839FBFE6CF20
:100CA000F0E0E0E0F1CF877FF8CF8B3210F40C94C6
:100CB0001C060895282F30E0F901E85BF141E0813E
:100CC000EE2309F1E13021F0F0F0E63098F00895DC
:100CD0004091010A28553141F90120812C5F81E0C2
:100CE00090E001C0880F2A95EAF7809584238093CD
:100CF000010A089580E1E89FF0011124E05AF54FC0
:100D000081818F7E81830895FF920F931F93CF93EC
:100D1000DF93082F10E0F801EE5DF041F0809FEFC7
:100D2000F916A1F0EB018B3210F40E945A06F8017B
:100D3000E45CF041E08180E2E89FF0011124FC5F77
:100D400080818F2159F0CD2B39F4F682DF91CF913C
:100D50001F910F91FF900895F582F8CFD801A85503
:100D6000B1418C91309771F08F3F61F07096E80F30
:100D7000F11D9FB7F8948081CD2B39F4877F808354
:100D80009FBFE4CFF0E0E0E0F4CF8860F8CF8B3293
:100D900010F40C9484060895CF92DF92EF92FF92A4
:100DA0000F931F93CF93DF93EC016A017B01022F16
:100DB0008989882339F0E881F9810288F389E02D57
:100DC000CE01099598898091E205892B8093E205EF
:100DD0001FB7F89460E070E281EA97E0A7019601FE
:100DE0000E94D85069017A018FEFC81AD80AE80A20
:100DF000F80AF694E794D794C794EC85FD8586812C
:100E00008D7F8683EC85FD8586818683198AA091F6
:100E100023110A2E000CBB0BA70196010E949F50C4
:100E200020E034E040E050E00E947550EC85FD8504
:100E3000C20ED31EE41EF51EC086D186EC85FD854C
:100E40000783EC85FD858681806C8683EC85FD8536
:100E50008581806885838E8562E070E00E945506FA
:100E60008F8561E070E00E94C7068F8561E070E0C9
:100E70000E9455061FBFDF91CF911F910F91FF90E8
:100E8000EF90DF90CF9008950F931F93CF93082F8B
:100E900010E0F801EE5DF041C081CF3FB9F08B3238
:100EA00010F40E945A06F801E45CF041E08180E20F
:100EB000E89FF0011124FC5F8085C82381E090E069
:100EC00009F480E0CF911F910F91089580E090E0A8
:100ED000F9CFE82FF0E0E05CF1418E30B8F480818A
:100EE0008F30B0F48093060681E0809308068091ED
:100EF0000B0680FFFCCF2FB7F894909110068091DD
:100F000011062FBF89279827892708953E97E7CF95
:100F10008FEF90E00895CF93DF938FB7F8942091EF
:100F2000492A30914A2A40914B2A50914C2AE0910B
:100F3000BA0A9091B60A90FF06C02F5F3F4F4F4FFD
:100F40005F4FE091BA0A8FBFA091532AB091542A03
:100F5000C091512AD091522A0E949450EC9F900146
:100F6000ED9F300D1124620F731F811D911DDF91C4
:100F7000CF9108958F929F92AF92BF92CF92DF92BE
:100F8000EF92FF924B015C010E948B076B017C0189
:100F9000A8EEB3E0A50194010E949450C60ED71E9E
:100FA000E81EF91EC616D706E806F90618F40E94D0
:100FB0008B07F8CF0E948B076C157D058E059F056A
:100FC000C8F3FF90EF90DF90CF90BF90AF909F90CD
:100FD0008F9008952FB7F8946091452A7091462A12
:100FE0008091472A9091482A2FBF08950F931F930D
:100FF000CF93DF938C01EB0180915C2890915D2869
:10100000A0915E28B0915F28892B8A2B8B2B51F4FD
:101010000E94EA0760935C2870935D2880935E28A5
:1010200090935F280130110539F0CF3FDC07A1F420
:1010300081E08093612806C0CF3FDC0741F481E066
:1010400080936028DF91CF911F910F910895C093F5
:101050006528D0936628F6CFC0936328D093642880
:10106000F1CF7F928F929F92AF92BF92CF92DF92F9
:10107000EF92FF920F931F93CF93DF93782EEB01A4
:101080007A010091B92D1091BA2DD8011496CD9006
:10109000DC9021E0C114D10409F420E0822E912CCF
:1010A000F80181819281DC01ED91FC91048CF58D38
:1010B000E02DA401D8016C91099588159905D1F40A
:1010C00087EBA82E8DE2B82EC501875B9D4288155F
:1010D000990570F4F80181819281DC01ED91FC9118
:1010E0000284F385E02D0995F50181935F01ECCF32
:1010F000CD2859F20091B72D10E002C01595079543
:101100007A94E2F7017011270E94EA07012B09F097
:1011100059C088809980AA80BB8081149104A10461
:10112000B10431F4688379838A839B8310E024C0FF
:101130001D811111FBCF681979098A099B096D324C
:1011400071408105910598F081E08D838F819885AC
:101150008230910508F459C08430910508F066C0CA
:101160002D81222309F46EC081E08E835FC08C81C3
:10117000811102C081E08C838F819885029702974C
:1011800090F4112381F0D70117968D919C911897B7
:101190000297029740F419968D919C911A97179691
:1011A0008D939C931897812FDF91CF911F910F9171
:1011B000FF90EF90DF90CF90BF90AF909F908F9077
:1011C0007F9008951C811123C1F02D81211114C03D
:1011D00088809980AA80BB80681979098A099B094F
:1011E00089889A88092C000CAA08BB0886169706DD
:1011F000A806B90608F4AACF10E01C821D821E8240
:10120000188219821A821B82B7CF89879A872D810B
:10121000222399F0019771F083E090E08F83988703
:101220000E94EA076B877C878D879E871111E5CF27
:1012300011E0A2CF82E090E0F1CF21E082278F83FE
:101240009887F4CF29853A8589879A872F833887AD
:10125000EDCFFC019085957081E0953009F080E03C
:101260000895CF92DF92EF92FF920F931F93CF9347
:10127000DF93EC0188858B7F8887E881F981019075
:10128000F081E02DCE010995182F88858695817013
:101290001817B9F00E94EA076A837B838C839D83C9
:1012A000888592E089278887888582FB882780F94E
:1012B000DF91CF911F910F91FF90EF90DF90CF9032
:1012C00008950E94EA07CA80DB80EC80FD80AB01B4
:1012D000BC014C195D096E097F098E819F81B0E0C8
:1012E000A0E0481759076A077B07F0F288858170EC
:1012F0001817D1F20E94EA076A837B838C839D834F
:10130000888591E08927846088870E94EA0709859B
:101310001A852B853C85601B710B820B930B6D87A7
:101320007E878F87988B0E94EA0769877A878B87E9
:101330009C87BACFCF93DF93EC011886E881F981BF
:101340000190F081E02D0995882319F0888583604C
:1013500088870E94EA076A837B838C839D83DF9161
:10136000CF910895862FBA010C945506FC0181890E
:1013700030E020E08B3218F40E9444079C0181E0A9
:10138000232B09F480E008950895EF92FF920F93C4
:101390001F93CF93DF937C01EB018B01040F151F8B
:1013A000C017D10759F0D701ED91FC910480F58168
:1013B000E02D6881C70109958993F2CFDF91CF9124
:1013C0001F910F91FF90EF9008950F931F93CF936C
:1013D000DF93EC018B018091C008E881F9810480E2
:1013E000F581E02D86FD13C0612FCE010995182FE0
:1013F000E881F9810480F581E02D602FCE01099507
:10140000082FC801DF91CF911F910F910895CE0150
:101410000995082FE881F9810480F581E02D612F7D
:10142000CE010995182FEDCF00006093C40880917C
:10143000C30887FFFCCF8091C40808958F929F92C4
:10144000AF92BF92CF92DF92EF92FF920F931F93D2
:10145000CF93DF93FC018085882319F081FF0EC0B4
:101460007894DF91CF911F910F91FF90EF90DF90D3
:10147000CF90BF90AF909F908F90089580FFF1CF55
:1014800082849384A484B584C12CD12C760110E08D
:101490009401A501B601C701A0E00E949C5599F1F5
:1014A000217030E040E050E060E070E080E090E0EB
:1014B0000E949C55D9F0D0E0C0E0103370F4C12FE9
:1014C000C695C695C69580E2C89FE0011124C05F0D
:1014D000DB4F812F8770C80FD11DCF01810F911D68
:1014E000DC0152968C919881892B88839401A50107
:1014F000B601C70101E00E94815549015A016B0103
:101500007C011F5FC5CF86849784A088B188C12CD9
:10151000D12C760110E29401A501B601C701A0E02B
:101520000E949C5509F49DCF217030E040E050E0CE
:1015300060E070E080E090E00E949C55D9F0D0E03F
:10154000C0E0103370F4C12FC695C695C695B0E2C1
:10155000CB9FE0011124C05FDB4F812F8770C80F44
:10156000D11DCF01810F911DDC0152968C91988184
:10157000892B88839401A501B601C70101E00E946F
:10158000815549015A016B017C011F5FC4CFFC01E9
:101590006F3F710581F1808581FD2DC0603271053D
:1015A0005CF581E090E002C0880F991F6A95E2F730
:1015B00080959095092E000CAA0BBB0B4285538594
:1015C0006485758584239523A623B7238287938713
:1015D000A487B58782859385A485B585892B8A2BB9
:1015E0008B2B49F486859785A089B189892B8A2B15
:1015F0008B2B09F4108608956052710981E090E008
:1016000002C0880F991F6A95E2F780959095092E80
:10161000000CAA0BBB0B4685578560897189842312
:101620009523A623B72386879787A08BB18BD2CF2C
:10163000FC016F3F7105E9F1603371051CF082E038
:101640008087089580858160808760327105C4F449
:1016500081E090E002C0880F991F6A95E2F7092E99
:10166000000CAA0BBB0B4285538564857585842BC2
:10167000952BA62BB72B82879387A487B5870895D0
:101680006052710981E090E002C0880F991F6A954D
:10169000E2F7092E000CAA0BBB0B46855785608923
:1016A0007189842B952BA62BB72B86879787A08BC8
:1016B000B18B0895E0ECF8E020812E7F2083FC01BF
:1016C00017820895E0ECF8E082818E7F828308958E
:1016D000E0ECF8E082818160828308950F9391E0CD
:1016E0009093422A1092412A60933F2A7093402A95
:1016F00040933E2A20933D2A10923C2A10923B2A86
:1017000000933A2A880F8093392A23E030E044E09E
:1017100050E080913E2A882341F02093372A30936D
:10172000382A8091392A8E7F0BC080913D2A8823E8
:1017300051F04093372A5093382A8091392A81609A
:101740008093A70808C080913E2A811104C080912F
:101750003D2A882311F38091412A8823E1F3809167
:10176000412A8330B1F280913D2A882321F0809173
:101770003B2A0F9108958091412A823031F08530C3
:1017800031F0813031F480E0F4CF81E0F2CF83E0BA
:10179000F0CF84E0EECFE0EAF8E0918590669187A3
:1017A00022E030E02093372A3093382A8093292A88
:1017B0001092282A089581E08093282A1092292ADD
:1017C00093E09093AA089091AB0891FF10C01092FB
:1017D000352AE091262AF091272A09958093342A08
:1017E00085E090E08093372A9093382A08951092EC
:1017F000362A8093332A86E090E0F4CF8F929F922E
:10180000AF92BF92CF92DF92EF92FF92CF93DF938E
:1018100060342DE0720723E08207910508F454C07C
:10182000611525E372072CE08207910508F445C095
:1018300060387F448241910508F046C0C8E7D0E097
:1018400020E432E44FE050E080901128909012287C
:10185000A0901328B0901428C501B4010E94D8505C
:1018600069017A018AE0C81AD108E108F108C501C6
:10187000B40120E432E44FE050E00E94D850DE0191
:101880000E94945028EE33E040E050E00E94D8508F
:10189000C21AD30AE40AF50AF694E794D794C794D7
:1018A000C092A608DF91CF91FF90EF90DF90CF908C
:1018B000BF90AF909F908F900895CCE2D1E020E848
:1018C0003AE146E050E0C0CFC8EED3E020EA36E887
:1018D00041E050E0B9CF6093242A7093252A0895FF
:1018E0006093222A7093232A0895E091242AF0918C
:1018F000252A309741F01092212A1092202A09952A
:101900008091202A089580E00895E091222AF091A4
:10191000232A309759F030911F2A20911E2A32171E
:1019200028F010921F2A80931E2A09940895089582
:10193000E0911F2A80911E2AE81730F4F0E0E25669
:10194000F64D808190E008958FEF9FEF089590917C
:101950001F2A80911E2A2FEF3FEF981748F4E92F96
:10196000F0E0E256F64D208130E09F5F90931F2A11
:10197000C901089580911E2A90911F2A891B990BF5
:101980000895CF92DF92EF92FF920F931F93CF9320
:10199000DF937C018A01EB016B01C40ED51ECC15CF
:1019A000DD0551F06991D701ED91FC910190F08135
:1019B000E02DC7010995F3CFC801DF91CF911F91A9
:1019C0000F91FF90EF90DF90CF9008952091202A03
:1019D00027FF08C021E030E0FC012283338390E040
:1019E00080E008958091212AE82FF0E0E25EF64D34
:1019F00060838F5F8093212A8093202A81E090E08A
:101A00000895DC01ED91FC91008CF18DE02D61E0F9
:101A100009940F938091372A9091382A0197A1F465
:101A20008091422A811112C0062F20E04091202A85
:101A30006EE179E280911D290E946E0B1092212A9D
:101A40001092202A0F91089580E0F8CF81E0F6CF20
:101A500060931D291092212A1092202A0895DC01FA
:101A6000ED91FC91048CF58DE02D21E009940F930C
:101A70008EE999E280932A2A90932B2A8091372A23
:101A80009091382A0197C9F48091422A811117C098
:101A9000FA014138510510F0E0E8F0E0022F862FFE
:101AA0002E2F40E070E060E00E946E0B10921F2A23
:101AB00080931E2A90E00F91089580E0F7CF81E097
:101AC000F5CFCB01BA010C94FE0BE0EAF8E01382EB
:101AD000168281E08583148611861092372A10922F
:101AE000382A089510921F2A10921E2A1092212A35
:101AF0001092202A8091372A9091382A892BD9F484
:101B000082E090E08093372A9093382A1092362A08
:101B10001092352A1092282A1092292A10921C29F4
:101B20001092332A660F6093AC0881EE8093A90867
:101B300081E08093A30885E79CE08093262A909318
:101B4000272A8EE199E280932C2A90932D2A85E80A
:101B50009CE08093312A9093322A8EE999E2809317
:101B60002E2A90932F2A80E88093302A089510928D
:101B70001F2A10921E2A1092212A1092202A809148
:101B8000372A9091382A892B41F562E070E086E18E
:101B90000E941C0662E070E087E10E941C068091B2
:101BA000E3058093E30581E090E08093372A9093EA
:101BB000382A10923B2A10923C2A1092422A109204
:101BC000412A81EC8093A30860EA76E881E090E006
:101BD0000E94FE0B81E08093A5080895CF93DF93C8
:101BE000EC018B818823D1F089819A81DC01ED9110
:101BF000FC910688F789E02D6881099589819A8191
:101C0000DC01ED91FC91028CF38DE02D099591E0C2
:101C1000811190E0892FDF91CF91089589819A8178
:101C2000DC01ED91FC910684F785E02D099581E0BA
:101C30008B83CE010E94EE0D982F8111D5CFEACF74
:101C4000FC01A5A1B6A18C9192A589238C93A5A195
:101C5000B6A18C9191A5892B8C930895DC01939664
:101C6000ED91FC919497908198968C918923808333
:101C70000895DC019396ED91FC919497908197964D
:101C80008C91892B80830895DC019196ED91FC91D4
:101C90009297908196968C91892380830895DC0198
:101CA0009196ED91FC919297908195968C91892BCC
:101CB00080830895CF92DF92EF92FF921F93CF938C
:101CC000DF93EC016A017B018DA981112BC08F2D5F
:101CD0009927AA27BB278093C4088091C30887FF50
:101CE000FCCFC701AA27BB278093C4088091C308F3
:101CF00087FFFCCFBB27AF2D9E2D8D2D8093C40871
:101D00008091C30887FFFCCFC092C4088091C308AC
:101D100087FFFCCFDF91CF911F91FF90EF90DF9075
:101D2000CF9008958130B1F410E2CE01F7FE0FC0DC
:101D30000E944F0ECE010E94390ECE010E942E0E3F
:101D4000CC0CDD1CEE1CFF1C115079F7E3CF0E9478
:101D5000440EF0CFEF8DF8A18F2D9927AA27BB272E
:101D60008083CE010E94200EEF8DF8A1C701AA2723
:101D7000BB278083CE010E94200EEF8DF8A1BB27E8
:101D8000AF2D9E2D8D2D8083CE010E94200EEF8DD4
:101D9000F8A1C082CE01DF91CF911F91FF90EF900B
:101DA000DF90CF900C94200EFF920F931F93CF9350
:101DB000DF93EC018B018DA9811112C01093C4082F
:101DC0008091C30887FFFCCF0093C4088091C308AB
:101DD00087FFFCCFDF91CF911F910F91FF90089566
:101DE0008130B1F490E1F92ECE0117FF0EC00E94B0
:101DF0004F0ECE010E94390ECE010E942E0E000F12
:101E0000111FFA94F110F0CFE5CF0E94440EF1CFEC
:101E1000EF8DF8A11083CE010E94200EEF8DF8A166
:101E20000083CE01DF91CF911F910F91FF900C9411
:101E3000200E0F931F93CF93DF93EC01162F8DA9E4
:101E400081110BC06093C4088091C30887FFFCCF49
:101E5000DF91CF911F910F910895813099F408E09F
:101E6000CE0117FF0CC00E944F0ECE010E94390E0A
:101E7000110FCE010E942E0E015091F7E9CF0E9462
:101E8000440EF3CFEF8DF8A16083CE01DF91CF91A7
:101E90001F910F910C94200ECF93DF93EC01ED8DE9
:101EA000FE8D80819CA989238083CE010E94190F19
:101EB000ED8DFE8D80819BA9892B8083DF91CF9151
:101EC00008958F929F92AF92BF92CF92DF92EF923E
:101ED000FF920F931F93CF93DF93EC0189AD9AADDF
:101EE000680F791F8BAD9CAD480F591F21503109E8
:101EF000260F371F4901B12CA12CCB01B0E0A0E087
:101F0000DC0199278827882A992AAA2ABB2A6801EE
:101F100081E0C81AD108C40ED51EF12CE12C70E066
:101F200060E0BA0155274427C42AD52AE62AF72AB1
:101F30006AE2CE010E944C0FB501A401CE010E94BD
:101F40005A0E6BE2CE010E944C0FB701A601CE01E2
:101F50000E945A0E6CE2CE01DF91CF911F910F913A
:101F6000FF90EF90DF90CF90BF90AF909F908F90B9
:101F70000C944C0FDC01D5962C91D59721110AC0F9
:101F80005F968D919C91DC01ED91FC910088F18927
:101F9000E02D099408950F931F93CF93DF93EC01E5
:101FA0002DA9211121C0DC018F8D98A1EC01E881C0
:101FB000F9810684F785E02D91960C919197929680
:101FC0001C91929793962C91939794963C91949709
:101FD00095964C91959796965C91969797966C915D
:101FE000979798967C910995DF91CF911F910F91CA
:101FF00008950F931F93CF93DF93EC018B010E9401
:10200000CB0F8FA987FD06C0EB8DFC8D80819AA92F
:1020100089238083ED8DFE8D80819CA98923808317
:1020200066E3CE010E94190FED8DFE8D80819BA984
:10203000892B80838DA9F8018230A1F06081CE01C7
:102040000E94190F8FA987FD06C0EB8DFC8D808142
:1020500099A9892B8083CE01DF91CF911F910F9198
:102060000C94BA0F88A9882349F360817181CE014D
:102070000E94D40EE7CFCF93DF931F92CDB7DEB788
:10208000FC0119826370668BDC01AD5BBF4F2C9144
:1020900030E011968C9190E0623031F06330C9F0FD
:1020A000613081F040EC498321AF32AF83AF94AF10
:1020B000BE016F5F7F4FCF010E94F90F0F90DF913C
:1020C000CF91089540EA498323AF34AF81AF92AFF7
:1020D000EFCF40E6F8CF0F931F93CF93DF931F927C
:1020E000CDB7DEB7FC0119826370668BDC01A85B9B
:1020F000BF4F2D913C91119712968D919C9162301A
:10210000D1F1633009F440C08F010C5B1F4F613087
:10211000F9F040EC4983AF014D5B5F4FDA014C9120
:1021200050E041AF52AFD8014C9150E043AF54AFB3
:102130002087318782879387BE016F5F7F4FCF01F2
:102140000E94F90F0F90DF91CF911F910F91089589
:1021500040EA4983D8014C9150E041AF52AFDF01D2
:10216000AA5BBF4F4C9150E043AF54AF22873387F7
:1021700080879187E1CFDF01AA5BBF4F4C9150E090
:1021800041AF52AF1196D0CF40E64983DF01A95B42
:10219000BF4F4C9150E041AF52AF1497E3CF1F9324
:1021A000CF93DF93EC01162FE881F9810284F38548
:1021B000E02D0995112371F06DADCE010E944C0FF9
:1021C000E881F9810688F789E02DCE01DF91CF9172
:1021D0001F9109946EADF1CFAF92BF92CF92DF9273
:1021E000EF92FF920F931F93CF93DF93EC0177FD54
:1021F00038C088859985681779079CF557FD31C0E7
:102200008A859B854817590764F569017A015B0146
:10221000E881F9810284F385E02DCE010995E881FA
:10222000F98102A4F3A5E02D01E010E021E030E007
:10223000A701B501CE010995B601CE010E94D40EC9
:10224000E881F9810688F789E02DCE01DF91CF91F1
:102250001F910F91FF90EF90DF90CF90BF90AF90C4
:102260000994DF91CF911F910F91FF90EF90DF9034
:10227000CF90BF90AF9008958F929F92AF92BF92F0
:10228000CF92DF92EF92FF920F931F93CF93DF9342
:10229000EC0149015701E881F98102A4F3A5E02D81
:1022A00009959401D8010E9470556B017C01C114FD
:1022B000D104E104F10409F481C08DA9811119C090
:1022C00081E0C81AD108E108F1088FEFC816D806D6
:1022D000E806F80609F472C0B092C4088091C308F9
:1022E00087FFFCCFA092C4088091C30887FFFCCF72
:1022F000E7CF813099F581E0C81AD108E108F108EB
:102300008FEFC816D806E806F80609F457C00B2D5B
:1023100018E0CE0107FF1CC00E944F0ECE010E94A4
:10232000390ECE010E942E0E000F115091F70A2D8A
:1023300018E0CE0107FF0FC00E944F0ECE010E9491
:10234000390ECE010E942E0E000F115091F7D3CFFF
:102350000E94440EE3CF0E94440EF0CFBA1016C084
:10236000CC0CDD1CEE1CFF1CEF8DF8A1B08281E0CF
:10237000C81AD108E108F1088FEFC816D806E80698
:10238000F806E1F0CE010E94200EF1CF81E0C81ADC
:10239000D108E108F1088FEFC816D806E806F8065C
:1023A00069F0EF8DF8A1B082CE010E94200EEF8D72
:1023B000F8A1A082CE010E94200EE8CFDF91CF913C
:1023C0001F910F91FF90EF90DF90CF90BF90AF9053
:1023D0009F908F9008958F929F92AF92BF92CF92CD
:1023E000DF92EF92FF920F931F93CF93DF934C01F5
:1023F000EB016A01590137FF07C0C9010196C80FF7
:10240000D91FB194A194B108F401A085B185CA1770
:10241000DB070CF058C017FF07C0C8010196C80EB3
:10242000D91E119501951109F40182859385C8166D
:10243000D9060CF048C0FE01EA0DFB1DAF0141506A
:10244000510957FD40C0B601600F711F9B0121501B
:10245000310937FD38C0D7FF03C05F01D0E0C0E0CD
:10246000D7FE03C08B01D12CC12C4A175B071CF08F
:102470005D01AC1ABD0A281739071CF08C010C1934
:102480001D09D401ED91FC910284F385E02DC40176
:1024900009959501A601BE01C4010E943C11D40119
:1024A000ED91FC910688F789E02DC401DF91CF9171
:1024B0001F910F91FF90EF90DF90CF90BF90AF9062
:1024C0009F908F900994DF91CF911F910F91FF9072
:1024D000EF90DF90CF90BF90AF909F908F90089536
:1024E000EF92FF920F931F932115310529F00115EB
:1024F000110511F00E94EB111F910F91FF90EF90C9
:1025000008958F929F92AF92BF92CF92DF92EF92F7
:10251000FF920F931F93CF93DF935C014B016A01EE
:10252000E90177FD52C0DC0118968D919C916817E6
:1025300079070CF04AC0209709F447C037FF07C05D
:10254000C9010196C80ED91ED195C195D109F501D1
:1025500082859385C816D906C4F5A6014C0F5D1F68
:102560009A012150310937FD30C0D7FE03C0EA017E
:10257000D12CC12C281739071CF0EC01CC19DD092E
:10258000D501ED91FC910284F385E02DC5010995FB
:1025900078018E0121E030E0A601B401C5010E945E
:1025A0003C11D501ED91FC910688F789E02DC5011C
:1025B000DF91CF911F910F91FF90EF90DF90CF901F
:1025C000BF90AF909F908F900994DF91CF911F9112
:1025D0000F91FF90EF90DF90CF90BF90AF909F90C2
:1025E0008F9008958F929F92AF92BF92CF92DF9279
:1025F000EF92FF920F931F93CF93DF935C016B01D8
:102600004A01E90157FD52C0DC011A968D919C9157
:10261000481759070CF04AC0209709F447C037FF04
:1026200007C0C9010196C80ED91ED195C195D1091F
:10263000F50180859185C816D906C4F5A6014C0F11
:102640005D1F9A012150310937FD30C0D7FE03C00C
:10265000EA01D12CC12C281739071CF0EC01CC1948
:10266000DD09D501ED91FC910284F385E02DC501D2
:102670000995780101E010E09E01A401B601C501B1
:102680000E943C11D501ED91FC910688F789E02D5F
:10269000C501DF91CF911F910F91FF90EF90DF90D7
:1026A000CF90BF90AF909F908F900994DF91CF9182
:1026B0001F910F91FF90EF90DF90CF90BF90AF9060
:1026C0009F908F900895EF92FF920F931F93CF9357
:1026D000DF9377FD32C0DC011896ED91FC916E1707
:1026E0007F075CF52115310541F137FF07C0F9017E
:1026F00031964E0F5F1F319521953109DC011A96F5
:10270000ED91FC914E175F07C4F4EA01C20FD31F8D
:10271000DE011197B7FD11C057FF03C09E0150E0C5
:1027200040E0AE17BF071CF09F01241B350B78015A
:10273000890121E030E00E943C11DF91CF911F918F
:102740000F91FF90EF900895EF92FF920F931F93D8
:10275000CF93DF9357FD31C0DC011A96ED91FC91C8
:102760004E175F0754F52115310539F137FF07C0C2
:10277000F90131966E0F7F1F319521953109DC01EA
:102780001896ED91FC916E177F07BCF4EB01C20F18
:10279000D31FDE011197B7FD10C077FF03C09E0164
:1027A00070E060E0AE17BF071CF09F01261B370BDF
:1027B000780101E010E00E943C11DF91CF911F9160
:1027C0000F91FF90EF9008958F929F92AF92BF92DA
:1027D000CF92DF92EF92FF920F931F93CF93DF93ED
:1027E00047012115310509F44BC00115110509F404
:1027F00047C037FF07C0F90131966E0F7F1F319533
:1028000021953109DC011896AD90BC906A157B05C5
:10281000BCF517FF07C0F80131964E0F5F1F1195E9
:1028200001951109DC011A96ED91FC914E175F0795
:102830003CF56B01C20ED31EE6012197D7FD20C0E7
:102840007A01E00EF11ED7011197B7FD19C077FF8D
:1028500003C0960170E060E057FF03C0870150E0BD
:1028600040E0CA15DB051CF09501261B370BAE179F
:10287000BF071CF08F01041B150B74010E943C1153
:10288000DF91CF911F910F91FF90EF90DF90CF904C
:10289000BF90AF909F908F900895EF92FF920F930B
:1028A0001F93CF93DF93EC0177FD22C08885998534
:1028B00068177907ECF457FD1BC08A859B8548177C
:1028C0005907B4F47901E881F98102A4F3A5E02D58
:1028D00001E010E021E030E0CE010995B701CE0122
:1028E000DF91CF911F910F91FF90EF900C94D40E38
:1028F000DF91CF911F910F91FF90EF900895DC0130
:10290000D7962C91D79727FD09C05B96ED91FC9146
:102910005C972081D1963C91232B20830C94BA0F95
:10292000CF93DF93EC010E94CB0F8FA987FD06C0E8
:10293000EB8DFC8D80819AA989238083DF91CF91D3
:1029400008950895FC016370668B848195812681CA
:102950003781613039F0633029F080879187228791
:1029600033870895208731878287938708952F9230
:102970003F924F925F926F927F928F929F92AF920F
:10298000BF92CF92DF92EF92FF920F931F93CF935C
:10299000DF93CDB7DEB76A97CDBFDEBF898F9A8F41
:1029A00069837A834A01D22E0F8318873701BC2CA2
:1029B000DC0159962D913C915A972115310509F06A
:1029C00012C118968D919C911997681779070CF090
:1029D000D4C11A968D919C91481759070CF0CDC11E
:1029E0004C2C512CB6E0CB9E600D711D11246B87D1
:1029F0007C87161617060CF0C0C1EA2DF0E0E987B7
:102A0000FA8793E0EE0FFF1F9A95E1F7EF87F88BB7
:102A1000CF01840F951F181619060CF0AEC1A98DB1
:102A2000BA8D58968C91811104C0BFEABD1508F487
:102A3000D394A98DBA8DED91FC9111970284F38501
:102A4000E02DCD010995B5E0DB9EC0011124E9819F
:102A5000FA81EB83FC83312C212C9C0128513D4FC2
:102A60002F8B388F4A2D50E04D8B5E8BEF89F88D80
:102A7000E20DF31D44918D829E82D12CC12C69817F
:102A80007A81620D731D698B7A8B842F90E08B8B1A
:102A90009C8BE98DFA8DA081B18140FF7FC0F1E070
:102AA000BF126CC0AF126AC01C96ED91FC912F81D1
:102AB0003885A4014C0D5D1D69897A89898D9A8DAF
:102AC0000995EB89FC89F595E7954E2F5FEFC51ABF
:102AD000D50A6D817E818D899E89680F791F6D83EE
:102AE0007E8398E0C916D10481F6AFEF2A1A3A0A1C
:102AF000EB81FC81E40DF51DEB83FC83F5E02F16E3
:102B0000310409F0B3CF2F81388526153705B9F088
:102B1000A98DBA8DED91FC91B1E0BB1254C0AB12FE
:102B200052C069817A816B5F7F4F0088F189E02D07
:102B3000830128E030E0A401898D9A8D0995A98D43
:102B4000BA8DED91FC9111970688F789E02DCD01A2
:102B50006A96CDBFDEBFDF91CF911F910F91FF909D
:102B6000EF90DF90CF90BF90AF909F908F907F902D
:102B70006F905F904F903F902F9009941E96ED912B
:102B8000FC91EF80F88409851A8592014D815E8160
:102B90006B817C81898D9A8D099593CF2F813885A2
:102BA0002615370509F48DCF31E0B31207C0A31203
:102BB00005C01C96ED91FC9193017BCF1E96ED9183
:102BC000FC917301E0CF6B857C85641975090684DF
:102BD000F785E02D73010F8518899201A401898D75
:102BE0009A8D0995ACCFF90134969491329745911D
:102BF0005491D91AB7E0DB9E400D511D1124F90103
:102C0000259134912B8B3C8BFA0125903490FA015D
:102C10003296749031963491398B32966490319615
:102C2000449041E04C1518F04A1508F07FC0662D1D
:102C3000062C000C770B6B837C83842D042C000CFA
:102C4000990B8D839E83A98DBA8DED91FC9111977F
:102C50000284F385E02DCD010995512CD12CC12C96
:102C6000EA2DF0E0E987FA872B2D30E02B873C87AF
:102C7000A401440D511D47FC5A954F8B588F698113
:102C80007A81660D711D67FC7A956D877E877989DB
:102C9000C71608F054CF2C2D30E04D815E81420FD5
:102CA000531FA985BA854A9FC0014B9F900D5A9F1B
:102CB000900D1124FC01E80DF91DEF87F88B852D8F
:102CC000612C4F89588D420F531F4D8B5E8B6714BB
:102CD00008F050C044244394480E877041F4C10169
:102CE0000196EB89FC89E20DF31DD4901C01D7FEFF
:102CF00019C0A98DBA8DED91FC91662D70E0B1E0FF
:102D0000BB1219C0AB1217C02D853E85620F731F11
:102D10000484F585E02D2F8138854D895E89898D64
:102D20009A8D0995DD0C6394842DD1CF1D821E826E
:102D30001B821C8288CF4B815C81640F751FAB8521
:102D4000BC856A9FC0016B9F900D7A9F900D1124E6
:102D500069817A81680F791F0684F785E02DEF80FD
:102D6000F88409851A859D014F855889898D9A8D2A
:102D70000995D8CF570CC3948ACF6A96CDBFDEBFD2
:102D8000DF91CF911F910F91FF90EF90DF90CF9047
:102D9000BF90AF909F908F907F906F905F904F907B
:102DA0003F902F9008958F929F92AF92CF92EF9283
:102DB000FF920F931F93CF93DF93EC01262F898D02
:102DC0009A8D009709F051C06A30D1F41C861D8697
:102DD0008D8948E0849F900111248E859F85820F04
:102DE000931F8E879F8781E090E0DF91CF911F91A5
:102DF0000F91FF90EF90CF90AF909F908F9008959C
:102E00006D3089F3CC88AD888F898823C1F08C859B
:102E10009D8536E0C39E800D911D112448855985FE
:102E20004817590764F44E855F851C861D8638E077
:102E3000A39EC0011124840F951F8E879F87EA8867
:102E4000FB88088919894E855F856C857D85CE0153
:102E50000E94B7142C898C859D8546E0249F800DA7
:102E6000911D11248C879D87BECF6A3069F41C8622
:102E70001D86FC013896E4912D898E859F85E29F01
:102E8000800D911D1124ADCF6D3009F4ACCFFC0144
:102E900034963491631708F4A6CF3296E491E6177E
:102EA00008F4A1CFFC01329685909490462F431BE5
:102EB000342F47E0349F800C911C1124F40132968A
:102EC00034913196E4913323A9F1EE2399F1CC8822
:102ED000F4013596E491AD884F89442301F10E2E1B
:102EE000000CFF0BE30FF11DCE9EA001CF9E500DF5
:102EF00011246C857D85460F571F68857985641779
:102F000075076CF44E855F851C861D86FC0138961E
:102F1000E491AE9E400D511D11244E875F87EA88D3
:102F2000FB88088919894E855F856C857D85CE0172
:102F30000E94B714F4013496E4912C898C859D8508
:102F4000E29F800D911D11248DCF6F927F928F9201
:102F50009F92AF92BF92CF92DF92EF92FF920F9328
:102F60001F93CF93DF93EC016B015A0139014801A4
:102F7000E881F9810284F385E02D0995E881F981E2
:102F80000288F389E02D87019301A501B601CE01E6
:102F90000995A501480D591D41505109E881F98154
:102FA0000288F389E02D9301B601CE010995E881ED
:102FB000F9810088F189E02D9401A501B601CE01C7
:102FC0000995C60CD71CB60161507109E881F981D9
:102FD0000088F189E02D9401A501CE010995E881D1
:102FE000F9810688F789E02DCE01DF91CF911F91FD
:102FF0000F91FF90EF90DF90CF90BF90AF909F9098
:103000008F907F906F9009946F927F928F929F9292
:10301000AF92BF92CF92DF92EF92FF920F931F93E6
:10302000CF93DF935C01EB016A014901380187010D
:10303000DC01ED91FC916217730719F564167506B2
:103040002CF0962D872D3A01C92ED82E96012619DF
:1030500037092F5F3F4F048CF58DE02DA301BE0192
:10306000C5010995DF91CF911F910F91FF90EF90CE
:10307000DF90CF90BF90AF909F908F907F906F9098
:1030800008954615570591F42617370724F0892D22
:103090004B01C22FD82F9E01281939092F5F3F4FAE
:1030A000068CF78DE02DA601B401DACF0284F385FA
:1030B000E02D0995D501ED91FC910488F589E02D6D
:1030C00083019401A601BE01C5010995D501ED91C9
:1030D000FC910688F789E02DC501DF91CF911F9102
:1030E0000F91FF90EF90DF90CF90BF90AF909F90A7
:1030F0008F907F906F900994EF92FF920F931F93A0
:10310000DC011A960D911C911B9718962D913C91FC
:103110001997ED91FC9100A0F1A1E02D7B0150E009
:1031200040E070E060E009951F910F91FF90EF90F3
:1031300008954F925F926F927F928F929F92AF927B
:10314000BF92CF92DF92EF92FF920F931F93CF9394
:10315000DF936C012B015A0139014801DC01ED912B
:10316000FC910284F385E02D0995E201640C751C45
:10317000D601ED91FC91C615D7055CF40088F18964
:10318000E02D87019401A501BE01C6010995219694
:10319000EFCF0688F789E02DC601DF91CF911F910F
:1031A0000F91FF90EF90DF90CF90BF90AF909F90E6
:1031B0008F907F906F905F904F9009948F929F9225
:1031C000AF92BF92CF92DF92EF92FF920F931F9335
:1031D000CF93DF93EC015B014A016901E881F9813A
:1031E0000284F385E02D099595012C0D3D1D21509C
:1031F0003109E881F9810488F589E02D780184019D
:10320000A401B501CE010995E881F9810688F78905
:10321000E02DCE01DF91CF911F910F91FF90EF90A4
:10322000DF90CF90BF90AF909F908F9009948F9236
:103230009F92AF92BF92CF92DF92EF92FF920F9345
:103240001F93CF93DF93EC015B014A016901780181
:10325000E881F9810284F385E02D0995C80CD91C19
:10326000860101501109E881F9810488F589E02D72
:103270009501A401B501CE010995E881F98106887F
:10328000F789E02DCE01DF91CF911F910F91FF9033
:10329000EF90DF90CF90BF90AF909F908F90099468
:1032A000EF92FF920F931F93DC01ED91FC9100A030
:1032B000F1A1E02D09951F910F91FF90EF900895D6
:1032C0000F931F93DC01ED91FC91068CF78DE02D9F
:1032D00009951F910F9108950F931F93DC01ED91B4
:1032E000FC91048CF58DE02D09951F910F910895A7
:1032F000DC01ED91FC910084F185E02D09942F9281
:103300003F924F925F926F927F928F929F92AF9275
:10331000BF92CF92DF92EF92FF920F931F93CF93C2
:10332000DF93CDB7DEB72697CDBFDEBF3C016A0184
:103330002D833E83EB82FC825801A41AB50AB7FEA6
:1033400003C0B194A194B1088D809E80861A970A1B
:1033500097FE03C09194819491088A149B045CF0B9
:10336000902F812F0D811E819D838E839C2D8D2D0D
:103370006B01692F782F0C151D055CF09D818E81E6
:103380006D837E83692F782F902F812F8601C92E20
:10339000D82E1601201A310A2B012D813E81421AA6
:1033A000530A57FE03C0519441945108710137FEEE
:1033B00003C03FEFE31AF30AF594E7948D819E81F1
:1033C000861797075CF5A1E0B0E0A983BA83C01621
:1033D000D1064CF1D301ED91FC910484F585E02DEB
:1033E0002B813C81A8016D817E818A149B041CF095
:1033F0004D815E81B801C3010995E418F508F7FE17
:103400000AC02D813E8189819A81280F391F2D8321
:103410003E83E20CF31C0F5F1F4FD9CF2FEF3FEF1E
:1034200029833A83D4CF2696CDBFDEBFDF91CF91DB
:103430001F910F91FF90EF90DF90CF90BF90AF90D2
:103440009F908F907F906F905F904F903F902F90C4
:103450000895089590E080E00895DC015A96ED917A
:10346000FC91309709F009940895DC015896ED918C
:10347000FC91309709F009940895DC015696ED917E
:10348000FC91309709F009940895DC015496ED9170
:10349000FC91309709F009940895362F642FDC01D0
:1034A0001E96ED91FC91309719F0422F832F0994CD
:1034B0000895DC01ED91FC910088F189E02D23E075
:1034C00030E00994CF92DF92EF92FF920F931F9317
:1034D000CF93DF93FC0127813085225031092230C0
:1034E000310530F58C010E94EA07F801C785D089C3
:1034F0000385148525853685601B710B820B930B24
:103500009E010D2E000C440B550B0E94D850AE01AD
:10351000D7FF02C04F5F5F4F559547956A01550F22
:10352000EE08FF0821E0C616D706E806F90608F0FF
:1035300020E0822FDF91CF911F910F91FF90EF90AC
:10354000DF90CF900895862F9091B12A9923A1F012
:103550006CE00E944A55E92FF0E0EE0FFF1FE65F96
:10356000F1418081918197FD07C080933528909328
:10357000362881E08093B32A0895FC0120813181AF
:1035800042815381FB0160817181828193810E941C
:1035900009510E94ED51CB010895CF92DF92EF9235
:1035A000FF920F931F93CF93DF936C019A018BE1EE
:1035B000869FE001879FD00D1124F12CE12C0BE1B7
:1035C00010E0AE01B6018BEB9DE20E947012EBEBB6
:1035D000FDE2C486D5862396C687D787DF91CF9133
:1035E0001F910F91FF90EF90DF90CF900895109270
:1035F0000D2910920E2910920F2910921029109265
:10360000CF2A1092D02A109238281092392810927E
:103610003A2810923B281092092910920A291092F8
:1036200007291092082908954F925F926F927F9216
:103630008F929F92AF92BF92CF92DF92EF92FF92C2
:103640000F931F93CF93DF93CDB7DEB72E97CDBFE8
:10365000DEBF8091452890914628029709F04FC11E
:103660002091E32A298381E082278093D22A0E9435
:103670008B074B015C013981332309F438C18091F8
:10368000A2289091A328A091A428B091A528A501D3
:103690009401281B390B4A0B5B0BCA01B9010E942C
:1036A000235269837A838B839C83209131283091C4
:1036B000322840913328509134280E94325320E020
:1036C00030E044EB52E40E947B5120E030E040E0E7
:1036D0005FE30E940A510E94ED516B01770FEE08E3
:1036E000FF080091442C1091452CD8018C918E7FBD
:1036F0008C938C918670823009F45FC0843051F0D5
:1037000081110FC044E0CC0CDD1CEE1CFF1C4A955F
:10371000D1F707C062E0F694E794D794C7946A950E
:10372000D1F780E090E0A1E0B0E08093522C90933C
:10373000532CA093542CB093552C97014427552714
:103740002B873C874D875E872093462C3093472CF0
:103750004093482C5093492CC701B60188279927DC
:1037600060934A2C70934B2C80934C2C90934D2C4F
:10377000232B242B252B09F444C0412C512C32013E
:103780006394A301920121503109410951092D830C
:103790003E834F8358876130710581059105A9F4F7
:1037A000C701B6010E94D8502B873C874D875E87A2
:1037B0004D805E806F807884E4CF53E0CC0CDD1CBC
:1037C000EE1CFF1C5A95D1F7ACCF60934A2C709336
:1037D0004B2C80934C2C90934D2C4092522C509219
:1037E000532C6092542C7092552C2B853C854D8522
:1037F0005E852093462C3093472C4093482C509361
:10380000492C8091522C9091532CA091542CB09122
:10381000552C0197A109B1098093522C9093532CF8
:10382000A093542CB093552C40914A2C50914B2C82
:1038300060914C2C70914D2C41155105610571051D
:1038400061F0415051096109710940934A2C50932C
:103850004B2C60934C2C70934D2C4091462C5091E6
:10386000472C6091482C7091492C40934E2C5093DA
:103870004F2C6093502C7093512C452B462B472B8B
:1038800021F480914A2C90914B2CD8011C968D9359
:103890009C931D971A961D921C921B978C91816088
:1038A0008C93C501B4010E9423526B017C0120E07E
:1038B00030E040EC5FE369817A818B819C810E94DA
:1038C00032539B01AC01C701B6010E940A5120E0AE
:1038D00030E04AE754E40E947B510E94F451609327
:1038E000DF2A7093E02A8093E12A9093E22A809263
:1038F000A2289092A328A092A428B092A5282E9640
:10390000CDBFDEBFDF91CF911F910F91FF90EF9060
:10391000DF90CF90BF90AF909F908F907F906F90EF
:103920005F904F9008958091452890914628892B6B
:1039300029F08091E32A882309F454C08091582A01
:103940009091592AA0915A2AB0915B2A0196A11D03
:10395000B11D8093582A9093592AA0935A2AB09364
:103960005B2A80911628909117284091582A5091EF
:10397000592A60915A2A70915B2A092E000CAA0BD1
:10398000BB0B481759076A077B0748F081E090E0B6
:103990008093D52A9093D62A8093D32A0895809134
:1039A0001628909117284091582A5091592A6091D1
:1039B0005A2A70915B2A97FD019695958795092E55
:1039C000000CAA0BBB0B481759076A077B0750F07E
:1039D0008091D52A9091D62A892B21F01092D52A50
:1039E0001092D62A08954F925F926F927F928F9293
:1039F0009F92AF92BF92CF92DF92EF92FF92CF93BE
:103A0000DF93EC016A017B01488459846A847B84DA
:103A10008C809D80AE80BF8020E030E0A901C30192
:103A2000B2010E9476518823A1F1A5019401C7013A
:103A3000B6010E9409510E94ED519B0177FF04C01D
:103A400022273327261B370BB901330F880B990B1D
:103A50000E9425529B01AC01C301B2010E94765124
:103A600087FF17C0CC82DD82EE82FF826C817D8170
:103A70008E819F81DF91CF91FF90EF90DF90CF906B
:103A8000BF90AF909F908F907F906F905F904F907E
:103A90000895488059806A807B80A301920160E08C
:103AA00070E080E89FE30E940951A50194010E9403
:103AB00032534B015C01A7019601C301B2010E9480
:103AC00032539B01AC01C501B4010E940A516C83C1
:103AD0007D838E839F83CACF8550883070F4E82F12
:103AE000F0E0EB58F24E0C946A55881D901D981D1D
:103AF000A01DA81DB01DB81DC01D60937E28709329
:103B00007F2860E77EE184E00E94310481E008952F
:103B100060938028709381286AE67EE185E0F4CF87
:103B2000609382287093832864E67EE186E0ECCF80
:103B300060938428709385286EE57EE187E0E4CF6A
:103B4000609386287093872868E57EE188E0DCCF63
:103B5000609388287093892862E57EE189E0D4CF5C
:103B600060938A2870938B286CE47EE18AE0CCCF46
:103B700060938C2870938D2866E47EE18BE0C4CF3F
:103B800060938E2870938F2860E47EE18CE0BCCF38
:103B9000DC01ED91FD918081ED91FD919081ED91A0
:103BA000FD916C9163708E2309F064609F2309F08E
:103BB0006860E5EEFDE1E60FF11D659565956D9395
:103BC0006D917D918D919D91099423C01AC012C071
:103BD00016C010C01EC009C014C013C006C019C052
:103BE00009C00DC007C00DC014C0625070408040B5
:103BF00090400BC0615070408040904006C06E5FA6
:103C000001C06F5F7F4F8F4F9F4F9E938E937E9328
:103C10006E9308958091A0289091A1280C94C81DBE
:103C200080919E2890919F280C94C81D80919C287B
:103C300090919D280C94C81D80919A2890919B2862
:103C40000C94C81D80919828909199280C94C81DB7
:103C500080919628909197280C94C81D8091942863
:103C6000909195280C94C81D80919228909193284A
:103C70000C94C81D80919028909191280C94C81D97
:103C800080918E2890918F280C94C81D80918C284B
:103C900090918D280C94C81D80918A2890918B2832
:103CA0000C94C81D80918828909189280C94C81D77
:103CB00080918628909187280C94C81D8091842833
:103CC000909185280C94C81D80918228909183281A
:103CD0000C94C81D80918028909181280C94C81D57
:103CE00080917E2890917F280C94C81D80917C281B
:103CF00090917D280C94C81D80917A2890917B2802
:103D00000C94C81D80917828909179280C94C81D36
:103D100080917628909177280C94C81DCF93DF93DB
:103D2000EC018B85823060F4F894CE010E94C81DAE
:103D30006F81788589859A857894DF91CF910895F0
:103D4000F894F6CF0F931F93CF93DF93EC01062FD8
:103D5000142F70E060E0802F0E94550661E070E053
:103D6000802F0E94C70670E060E0812F0E945506F8
:103D700061E070E0812F0E94C706802F90E0FC0177
:103D8000E45CF041A081A63008F04EC020E2A29F82
:103D9000D0011124BC5F9D01285F3F4F28833983E8
:103DA0008E5D9041FC0140814C83812F90E0FC01AD
:103DB000E45CF041E08170E060E0E63030F420E265
:103DC000E29FF0011124BF017C5F9B01285F3F4F00
:103DD0002A833B838E5D9041FC0130813D831F82AD
:103DE000188619861A868BE39FE10197F1F71896DA
:103DF0002C91242381E009F480E0FB01908593233A
:103E000009F082608E83BE01802F0E946C1D8B871B
:103E1000BE01812F0E946C1D9B85890F8B87DF91CE
:103E2000CF911F910F910895B0E0A0E0B4CF8F9291
:103E30009F92AF92BF920F931F93CF93DF93CDB713
:103E4000DEB7A197CDBFDEBF19A2423008F44AE029
:103E50008E010F5D1F4F842E912CB12CA12CA5013A
:103E600094010E94D850E62FB901CA01EA302CF51E
:103E7000E05DD801EE938D01232B242B252B79F7C0
:103E800090E080E0109769F0FD0101900020E9F7D3
:103E90003197AF014A1B5B0BBD018BEB9DE20E948A
:103EA0008F05A196CDBFDEBFDF91CF911F910F91FE
:103EB000BF90AF909F908F900895E95CDACFCF923A
:103EC000DF92EF92FF92CF93DF936B017C016DE263
:103ED0008BEB9DE20E94D316EC0166277727CB017E
:103EE0006C197D098E099F094AE00E94171F8C0FEB
:103EF0009D1FDF91CF91FF90EF90DF90CF900895BD
:103F0000009769F0FC0101900020E9F73197AF01BB
:103F1000481B590BBC018BEB9DE20C948F0590E084
:103F200080E0089540EA50E062E070E090E080E0D8
:103F30000E94CD1A0E94EA078091E72A9091E82A10
:103F40008093E52A9093E62A863091059CF488E9CF
:103F50009FEE0E94801F8091E52A9091E62A86308C
:103F6000910510F5880F991FFC01EC56F1418081F5
:103F7000918115C089309105A9F740EA50E062E0CF
:103F800070E090E080E00E94CD1A8DE99FEE0E94E3
:103F9000801F8091E42A811104C082E090EF0C948C
:103FA000801F84E99FEEFBCF08958F929F92AF927E
:103FB000BF92CF92DF92EF92FF920F931F93CF9316
:103FC000DF937C016B018A012417350710F030E084
:103FD00020E0E901219740EF50E063E070E08AE0E3
:103FE00090E00E94CD1AC7010E94801F99E1E92E3E
:103FF0009CEFF92E8091682A9091692A0E948E1E6A
:104000004B01940121703327232B11F594012E19B4
:104010003F0912161306DCF16E157F05C9F08FEF0C
:104020009FEFC80FD91FD7FF35C0C00FD11F44E67F
:1040300050E063E070E080EA90E00E94CD1AFE015B
:10404000EE0FFF1FEC0DFD1D808191810E94801FEE
:1040500080916C2A90916D2A0E943109E0916C2A1E
:10406000F0916D2A808580FD10C082FF0EC0CE01C8
:10407000DF91CF911F910F91FF90EF90DF90CF9044
:10408000BF90AF909F908F9008957401B3CF81E05F
:1040900090E0C7CFC017D10754F2C01BD10BC7CFD8
:1040A000CF92DF92EF92FF922091B92A211156C050
:1040B00041110EC0C090A628D090A728E090A82853
:1040C000F090A928C616D706E806F90609F446C0F6
:1040D0006B017C01C092A628D092A728E092A82864
:1040E000F092A9284CE350E064E070E08CE390E0AB
:1040F0000E94CD1A8091452890914628892B79F00D
:1041000081EBC81684E0D806E104F10444F088EAA3
:104110009FEEFF90EF90DF90CF900C94801FF7FE02
:1041200017C0C701B6010E945F1F20E030E040E8E1
:104130005FE360913128709132288091332890910B
:1041400034280E947651882349F08AEA9FEEE1CF15
:104150004AE0C701B6010E94171FE7CFFF90EF901A
:10416000DF90CF900895BC01990F880B990B97FDB4
:104170000C945F1F4AE00C94171FCF93DF93873F87
:104180002FEF920724F4DF91CF910C94B320EC0130
:1041900097FF06C08FEA9FEE0E94801FCE01F3CFEB
:1041A0008CEA9FEECA30D105BCF78EEA9FEE2097CD
:1041B00099F781EB9FEEDF91CF910C94801F7F9256
:1041C0008F929F92AF92BF92CF92DF92EF92FF9227
:1041D0000F931F93CF93DF93062F5A01882361F02B
:1041E00040EA50E061E070E090E080E00E94CD1A8B
:1041F00085EB9FEE0E94801F21E8C22E2AE2D22E7C
:10420000D0E0C0E010E03AE2732E011169C0AC16B4
:10421000BD0609F469C080910228909103288C178B
:104220009D0729F5EE24EA94FE2CF601808091800A
:1042300063E070E0C430D10514F462E070E04AE25B
:1042400050E0CE01837099279C01729EC001739E3D
:10425000900D11240E94CD1AE092CD2DF092CE2D1A
:10426000E092CB2DF092CC2DC4010E94BD20111103
:1042700007C011E0F60180819181892B09F410E0DB
:104280002196F2E0CF0ED11CC830D10509F0BDCF88
:104290008FEF9FEF8093CD2D9093CE2D8093CB2DDC
:1042A0009093CC2D112341F0809145289091462880
:1042B00011E0892B09F410E01093E32AA092022860
:1042C000B0920328DF91CF911F910F91FF90EF9053
:1042D000DF90CF90BF90AF909F908F907F90089588
:1042E000AC16BD0609F09ECF87EEE82E89EFF82EBA
:1042F0009CCF8F929F92AF92BF92CF92DF92EF921C
:10430000FF920F931F93CF93DF93962E7A0188230A
:1043100061F040EA50E061E070E090E080E00E94EF
:10432000CD1A82EC9FEE0E94801F81E2C82E88E2A7
:10433000D82ED0E0C0E09AE2892E911051C0EC1640
:10434000FD0609F451C080910428909105288C172E
:104350009D0721F50FEF1FEFF601A080B18063E00C
:1043600070E0C430D10514F462E070E04AE250E03D
:10437000CE01837099279C01829EC001839E900D7F
:1043800011240E94CD1A0093CD2D1093CE2D0093B1
:10439000CB2D1093CC2DC5010E94BD20219632E07B
:1043A000C30ED11CC830D10541F68FEF9FEF80932B
:1043B000CD2D9093CE2D8093CB2D9093CC2DE0924C
:1043C0000428F0920528DF91CF911F910F91FF9063
:1043D000EF90DF90CF90BF90AF909F908F90089517
:1043E000EC16FD0609F0B6CF07EE19EFB5CFEF9248
:1043F000FF920F931F93CF93DF930097A9F0409103
:104400004728509148286091492870914A284D3D8D
:1044100055406105710544F0209100283091012834
:104420002F3F3F4F09F450C02091D42D3091D52D0E
:10443000232B51F42091C92D3091CA2D2A5F3F4F73
:104440002093C92D3093CA2D2FED32E02093D42D27
:104450003093D52D1816190624F5EC0180914728C4
:1044600090914828A0914928B0914A288D3D9540C7
:10447000A105B10584F1E0901329F09014290FE310
:1044800010E028E330E048E350E066EB70E08BEBAF
:104490009DE20E94EB118FEF9FEF80930028909395
:1044A00001288091D42D9091D52D892B49F08091B0
:1044B000C92D9091CA2D06978093C92D9093CA2D2E
:1044C0001092D42D1092D52DDF91CF911F910F9185
:1044D000FF90EF90089580910028909101288C170B
:1044E0009D07F9F2E0901A29F0901B290FE310E0E4
:1044F00028E330E048E350E066EB70E08BEB9DE2B0
:104500000E94EB118CEB90E08093C72D9093C82D07
:104510008EE690E08093C92D9093CA2DCE010E9423
:10452000B320C0930028D0930128BBCFCF93DF9353
:10453000EC014CE050E061E070E080EC90E00E9423
:10454000CD1A1C161D062CF4CE01DF91CF910C94D0
:10455000B320DF91CF9108951F93CF93DF93182F4E
:104560008091C02AC6E0D0E081110AC08091B12AB2
:10457000C0913C28D0913D28882311F0C7E0D0E0BD
:104580008FEF9FEF8093CD2D9093CE2D8093CB2DE9
:104590009093CC2D82E08093CF2D8093D02D40EA54
:1045A00050E0C930D10509F05DC062E070E090E0F4
:1045B00080E00E94CD1A8DE99FEE0E94801F8091BD
:1045C000E42A81114CC082E090EF0E94801F84EBAE
:1045D00090E08093C72D9093C82DCEE1D0E0C0939A
:1045E000C92DD093CA2D8DEC9FEE0E94801F8CECBC
:1045F00090E08093C72D9093C82DC093C92DD09380
:10460000CA2D8FEC9FEE0E94801F80913E289091D2
:104610003F280E9496221123D9F040EA50E063E03F
:1046200070E090E080E00E94CD1A81ED9FEE0E9444
:10463000801F49E150E063E070E084E890E00E9470
:10464000CD1A8091952A9091962A01960E94B320C6
:1046500090E080E0DF91CF911F910C94F72184E9E5
:104660009FEEB3CF61E070E090E080E00E94CD1A51
:10467000CC0FDD1FCC56D14188819981A6CF809186
:10468000F02C9091F12C0297029750F480916028C1
:104690008823C9F150E040E061E081E00E94DF2022
:1046A0008091DD2C9091DE2C0297029750F480913E
:1046B0006128882389F150E040E061E081E00E94B8
:1046C000792180916228882329F081E00E94AC2220
:1046D0000E94921F10925C2810925D2810925E2812
:1046E00010925F2810926028109261288FEF9FEF40
:1046F000809363289093642880936528909366281C
:10470000109262280895409165285091662857FDBF
:10471000C7CF61E080E0C2CF409163285091642808
:1047200057FDCFCF61E080E0CACFCF93DF934091B8
:10473000B82D21E030E0D90102C0AA0FBB1F8A9535
:10474000E2F7CD016230E1F4842B8093B82DC09163
:10475000B92DD091BA2D8C819D81892BA1F08981B1
:104760009A81DC01ED91FC910688F789E02D688142
:10477000099568EB7DE2CE01DF91CF910C94600446
:1047800080958423E2CF80E0DF91CF910895CF938D
:10479000DF934091B82D21E030E0D90102C0AA0F8B
:1047A000BB1F8A95E2F7CD016623E1F0842B80934D
:1047B000B82DC091B92DD091BA2D8C819D81892BB6
:1047C000A1F089819A81DC01ED91FC910688F7893D
:1047D000E02D6881099568EB7DE2CE01DF91CF91F4
:1047E0000C94600480958423E2CF80E0DF91CF9128
:1047F0000895FF920F931F93CF93DF93F62E20918E
:10480000402830914128AC01421B530B281739072F
:1048100014F59A018093402890934128E90121974B
:104820008091AF2A882329F070E060E080E10E9447
:10483000840610E000E061E070E080E10C171D07E5
:1048400074F40E94840670E060E080E10E948406B7
:104850000F5F1F4FF0CF9A01285F3F4FDBCF0E94C1
:1048600084060E948B076093AB2A7093AC2A8093D6
:10487000AD2A9093AE2AC1E0C093AF2AFF2031F059
:1048800061E085E00E94C723C093B02A8091402850
:10489000909141280196DF91CF911F910F91FF9048
:1048A0000C94F721CF92DF92EF92FF920F931F9318
:1048B000CF93DF93EC01088119816A817B81601BB2
:1048C000710B072E000C880B990B0E9425529B013F
:1048D000AC0160E070E080EC91E40E947B516B01E0
:1048E0007C0168857985601B710B072E000C880B95
:1048F000990B0E9425529B01AC01C701B6010E9491
:1049000032530E94EF530E94ED51CB0197FF02C03A
:104910000C96FCCF6CE070E00E945655FC01EE0F47
:10492000FF1FE85DF141808191810197DF91CF9177
:104930001F910F91FF90EF90DF90CF9008954F92CD
:104940005F926F927F928F929F92AF92BF92CF921F
:10495000DF92EF92FF920F931F93CF93DF93CDB728
:10496000DEB72E97CDBFDEBFC0903128D090322861
:10497000E0903328F0903428BC0104970CF0B2C0CA
:104980006F5F7F4F072E000C880B990B0E942552FA
:104990009B01AC0160E070E080E89FE30E947B51E6
:1049A0006093AA287093AB288093AC289093AD288D
:1049B00020914528309146282230310561F421E0CC
:1049C0002983A70196010E947651811101C01982A5
:1049D00039813093AE288090AA289090AB28A0907F
:1049E000AC28B090AD2841E04983A7019601C501EC
:1049F000B4010E947651811101C0198259815093EE
:104A00006A2AA7019601C501B4010E947651882344
:104A100009F466C18091AE28811162C1809231286B
:104A200090923228A0923328B092342860910A28BC
:104A300070E090E080E00E942552A50194010E9460
:104A400032530E94ED51AB018091112990911229AE
:104A5000BA010E9456558093112990931229809390
:104A60000B2990930C2960914728709148288091D8
:104A7000492890914A280E94255269837A838B8322
:104A80009C839B01AC0160EC71EE84E69CE40E9487
:104A90007B51A50194010E94325320E030E044EBA9
:104AA00052E40E947B510E94EF530E94F4516B012B
:104AB0007C010091442C1091452CD8018C918E7F63
:104AC0008C938C918670823009F470C08430D9F058
:104AD000811120C044E0CC0CDD1CEE1CFF1C4A956B
:104AE000D1F718C063507109072E000C880B990B81
:104AF0000E9425526093AA287093AB288093AC281B
:104B00009093AD2868CF62E0F694E794D794C79469
:104B10006A95D1F780E090E0A1E0B0E08093522C5C
:104B20009093532CA093542CB093552C9701442769
:104B300055272B873C874D875E872093462C3093E3
:104B4000472C4093482C5093492CC701B601882725
:104B5000992760934A2C70934B2C80934C2C909304
:104B60004D2C232B242B252B09F444C0412C512CF4
:104B700032016394A3019201215031094109510985
:104B80002D833E834F8358876130710581059105E0
:104B9000A9F4C701B6010E94D8502B873C874D87E6
:104BA0005E874D805E806F807884E4CF53E0CC0CCC
:104BB000DD1CEE1CFF1C5A95D1F7ACCF60934A2C3C
:104BC00070934B2C80934C2C90934D2C4092522CF4
:104BD0005092532C6092542C7092552C2B853C850E
:104BE0004D855E852093462C3093472C4093482C6E
:104BF0005093492C8091522C9091532CA091542C7D
:104C0000B091552C0197A109B1098093522C909332
:104C1000532CA093542CB093552C40914A2C509176
:104C20004B2C60914C2C70914D2C41155105610518
:104C3000710561F0415051096109710940934A2C95
:104C400050934B2C60934C2C70934D2C4091462CE0
:104C50005091472C6091482C7091492C40934E2CD8
:104C600050934F2C6093502C7093512C452B462B16
:104C7000472B21F480914A2C90914B2CD8011C9603
:104C80008D939C931D971A961D921C921B978C9145
:104C900081608C938091452890914628892B01F55D
:104CA000A501940169817A818B819C810E947B514D
:104CB0000E94ED5140E02E96CDBFDEBFDF91CF9137
:104CC0001F910F91FF90EF90DF90CF90BF90AF902A
:104CD0009F908F907F906F905F904F900C9450209A
:104CE0002E96CDBFDEBFDF91CF911F910F91FF9028
:104CF000EF90DF90CF90BF90AF909F908F907F907C
:104D00006F905F904F9008950F931F93CF93DF9311
:104D10008091E72A9091E82A88309105A9F440EA29
:104D200050E061E070E090E080E00E94CD1A8CEDF0
:104D30009FEE0E94801F1092402810924128DF9120
:104D4000CF911F910F9108951092B12A1092C02A0D
:104D5000863091050CF04DC08091E52A9091E62AAD
:104D600080933C2890933D2882309105D1F481E0D6
:104D70008093422880E00E94AC228091B12A811168
:104D800004C08091C02A8823D1F240EA50E062E05A
:104D900070E090E080E0DF91CF911F910F910C9433
:104DA000CD1A049739F70CE318E2C8E0D0E00E946E
:104DB000914FBE010E945655D8015E962D913C91AF
:104DC0005F97FC01EE0FFF1FE45BF74D808191813F
:104DD0005E968D939C935F97332720833183219731
:104DE00002501109209719F7109243281092442875
:104DF000C1CF21E08730910509F020E02093B12A4E
:104E000021E08630910509F020E02093C02A09971F
:104E100009F0B0CF8091E42A91E089278093E42AB9
:104E200040EA50E062E070E090E080E00E94CD1A3D
:104E30008DE99FEE0E94801F8091E42A81111AC0A3
:104E400082E090EF0E94801F809145289091462833
:104E5000892B61F08091E42A882349F0209145282C
:104E60003091462881E02130310509F080E08093BF
:104E7000E32A80CF84E99FEEE5CF20914528309149
:104E800046282230310509F04BC02091552A309137
:104E9000562A1216130624F48217130609F040C08E
:104EA000842F90E024E0959587952A95E1F7877007
:104EB000613161F0623129F1603191F590E0019644
:104EC00080933E2890933F280C949622863040F59C
:104ED00090E02091E72A3091E82A8217930701F1A8
:104EE0008093E72A9093E82A8093E52A9093E62A14
:104EF00080916A2A882319F010926A2A08950C94E6
:104F00008426873069F0282F30E0843020F0C901F2
:104F100003970C949F2487E090E0821B930BF9CFBA
:104F20000895CF93DF9380913C2890913D28823063
:104F30009105E1F150F4C0913E28D0913F2821978E
:104F40000197C1F0D0E0C0E015C0C0914C28D091CD
:104F50004D288430910571F00597A1F70E94914F7B
:104F6000892F990F990B60913E2870913F280E94DC
:104F70005655EC01109243281092442860E0CE016F
:104F80000E94F9238091DD2C9091DE2C01970297ED
:104F900088F4CC0FDD1FCF5DD74D88819981809338
:104FA000A92A9093AA2ADF91CF91089581E0809356
:104FB0004228C8CF81E090E0F2CF0F931F93CF93A8
:104FC000DF938091E42A8823A9F088E790E080931A
:104FD00016289093172881E08093572A80914B28B8
:104FE0008823B1F181E08093B22ADF91CF911F91A4
:104FF0000F9108958091F02C9091F12C01970297D8
:1050000068F7C0914028D0914128CE01029608E06F
:1050100010E0B8010E945655FC01EE0FFF1FEF573C
:10502000F54D20813181265A3F4FCE010196B801BE
:105030000E945655FC01EE0FFF1FEF57F54D808182
:105040009181281B390B2093162830931728C6CF3F
:10505000DF91CF911F910F910C9491278091E32ABA
:10506000811122C08091452890914628019721F412
:105070008091D12A81110AC08091452890914628BB
:10508000029771F48091D22A882351F08091B22A3C
:10509000882359F01092B22A0E9491271092B32AC5
:1050A0001092D12A1092D22A089581E08093B32AD7
:1050B000F7CF0C9444560E94CD56CF92DF92EF92D8
:1050C000FF920F93FC01C12CB9E0DB2EBDE3EB2E68
:1050D000F12CC082D182E282F3821482158281E0B7
:1050E00090E086839783C0901128D0901228E0909A
:1050F0001328F0901428F694E794D794C79490E07E
:105100004C155D056E057F0540F4F694E794D79441
:10511000C7949F5F9630A1F797E004600187892FBD
:105120008095A82FA170B0E084E0AA0FBB1F8A95DC
:10513000E1F791629A2B80E0232B09F480E4982B0D
:1051400090870F91FF90EF90DF90CF9008950F938D
:105150001F93CF93DF93CDB7DEB72A97CDBFDEBFC6
:105160008C01FC01878181110CC01086118612868A
:1051700013861486158616861786108A118A81E092
:1051800087838091E305F8019681892B8093E3055D
:1051900061E070E083810E94550661E070E0F801F3
:1051A00084810E9455068091C10884608093C10863
:1051B0008091C00881628093C00840915C2C50911E
:1051C0005D2C60915E2C70915F2C0091602C209181
:1051D000622C3091632CCE0101960E945D28998546
:1051E0008A859093C0088093C1082A96CDBFDEBF00
:1051F000DF91CF911F910F910895CF92DF92EF929F
:10520000FF920F931F93CF93DF93EC016A017B0111
:10521000C114D104E104F10439F4C12C88E4D82E7E
:1052200088EEE82EFF24F394FE01FF96C082D1821F
:10523000E282F38281E28DAF80E28EAF36961081FA
:105240008FA987FD09C061E070E00E94550661E00A
:1052500070E08FA90E94C70661E070E088AD0E94EF
:10526000550661E070E088AD0E94C7068DA98111E6
:105270004DC0C9A2DAA2EBA2FCA2812F90E08DA3BF
:105280009EA381E090E08FA398A7812F90E0B0E0EB
:10529000A0E089A79AA7ABA7BCA78F8D98A180573C
:1052A0009C4221F480E79CE20E94A7288EA987FDFA
:1052B00086C061E070E00E94550661E070E08EA952
:1052C0000E94C70664E670E080E090E00E94BA07A2
:1052D00070E060E08EA90E94C70664E670E080E09E
:1052E00090E00E94BA0761E070E08EA90E94C706B4
:1052F00068EC70E080E090E0DF91CF911F910F911A
:10530000FF90EF90DF90CF900C94BA070CE31FEE64
:10531000F12C8130E1F461E070E08AA50E9455062D
:1053200070E060E08AA50E94C70661E070E08CA58D
:105330000E94550670E060E08CA50E94C7068BA510
:1053400087FDB4CF70E060E00E945506AFCFF80152
:1053500081918F01863080F5F0E28F9FC00111248A
:105360009C5F04962F8D38A12817390751F461E00E
:1053700070E08F2D0E94550670E060E08F2D0E9436
:10538000C706F39426E1F212E2CF61E070E08EA549
:105390000E94550661E070E08EA50E94C7068FA5A9
:1053A00087FD84CF61E070E00E94550661E070E007
:1053B0008FA50E94C7067ACF90E080E0D2CFDF9120
:1053C000CF911F910F91FF90EF90DF90CF900895B4
:1053D0005F926F927F928F929F92AF92BF92CF9285
:1053E000DF92EF92FF920F931F93CF93DF93CDB78E
:1053F000DEB76297CDBFDEBF3C010B871C872D87D0
:105400003E87042F4F87588B698B7A8B29893A897D
:105410004B855C856D857E85CE0101960E945D2859
:1054200059841A85D30118968C91882319F081FF2D
:1054300018C0F8945092C0081093C1086296CDBF6E
:10544000DEBFDF91CF911F910F91FF90EF90DF9022
:10545000CF90BF90AF909F908F907F906F905F9014
:10546000089580FFE7CFF30182849384A484B584F8
:10547000C12CD12C7601B0E09401A501B601C70181
:10548000A0E00E949C55A9F1217030E040E050E07E
:1054900060E070E080E090E00E949C55E9F090E0D0
:1054A00080E0B03370F48B2F869586958695F0E278
:1054B0008F9FC0011124805F9B4F2B2F2770820F7D
:1054C000911DFC01408193012B0F311DF901428B8D
:1054D000FC012081287F20839401A501B601C7012A
:1054E00001E00E94815549015A016B017C01BF5FB7
:1054F000C3CFD3011E968D909D90AD90BC905197D7
:10550000C12CD12C7601B0E29401A501B601C701EE
:10551000A0E00E949C5509F48DCF217030E040E05E
:1055200050E060E070E080E090E00E949C55E9F07F
:1055300090E080E0B03370F48B2F86958695869549
:10554000E0E28E9FC0011124805F9B4F2B2F2770BC
:10555000820F911DFC01408193012B0F311DF90138
:10556000428BFC012081287F20839401A501B60194
:10557000C70101E00E94815549015A016B017C017C
:10558000BF5FC2CFFF920F931F93CF93DF938C0126
:10559000EB01F8800E944550F81621F06F2DC801EC
:1055A0000E944D50CE01DF91CF911F910F91FF903E
:1055B00008950F931F93CF93DF938C01EB010E940B
:1055C00045508883C80101960E9445508983CE01C9
:1055D000DF91CF911F910F910895FF920F931F9329
:1055E000CF93DF93EC018B01FB01F0800E944550CB
:1055F000F81621F06F2DCE010E944D50F801F18078
:105600002196CE010E944550F81621F06F2DCE0153
:105610000E944D50C801DF91CF911F910F91FF90D3
:105620000895CF93DF93C0E1D0E0BE016F5E774D68
:10563000CE010E94ED2A2296C032D105B1F7DF914A
:10564000CF910895CF93DF93C4E2D0E0BE01635AB7
:10565000754DCE010E94ED2A2296C433D105B1F7D3
:10566000DF91CF910895CF93C62F80934B282AE5E1
:1056700030E0209316283093172861E0682784E0F3
:105680000E94C72360914B2870E081E10E9484064C
:10569000CC2391F00E94DD278091912A81110E94F4
:1056A000222B8091922A81110E94112B1092922A12
:1056B0001092912ACF9108958091E42A882361F372
:1056C00088E790E080931628909317281092572A25
:1056D000E3CF8091452890914628029721F460E01D
:1056E00080E00C94332B08958091452890914628B2
:1056F000029771F40E94F71A8FEF9FEF80931129A0
:105700009093122960E081E00E94332B0C94141BCB
:1057100008958091452890914628029791F40E941F
:10572000F71A8FEF9FEF809311299093122980939E
:105730000B2990930C2961E081E00E94332B0C949B
:10574000141B089590E00C944550882349F086E09E
:105750000E94A22B91E0811101C090E09093152945
:10576000809115292FE130E0882311F020E038EFF7
:1057700020931A2930931B2920EE3FEF882311F044
:105780002FEF3FEF2093182930931929811107C07B
:105790008AE090E08093132990931429089580E083
:1057A00090EAF8CF6F927F928F929F92AF92BF92C2
:1057B000CF92DF92EF92FF920F931F93CF93DF93DD
:1057C000CDB7DEB7CA54D109CDBFDEBFD82E81E038
:1057D0000E94A52B1092B92A70E060E08BEB9DE24D
:1057E0000E947C188091152861E0811163E08BEBA9
:1057F0009DE20E946B10E0901A29F0901B290DE1A8
:1058000010E020EF30E050E040E070E060E08BEB33
:105810009DE20E94EB118FEF9FEF8093CD2D90932F
:10582000CE2D8093CB2D9093CC2D8CE390E0809364
:10583000C72D9093C82D85E090E08093C92D90935B
:10584000CA2D82E08093CF2D8093D02D87EE9FEEDE
:105850000E94801FDD2009F413C28AE090E080934B
:10586000C72D9093C82D8EE190E08093C92D909321
:10587000CA2D82EF9FEE0E94801F68EE73E080E0E9
:1058800090E00E94BA0780E1E8EAFDEEDE01D396DF
:1058900001900D928A95E1F7FE01B39680E1DF0158
:1058A0001D928A95E9F77E01B3E3EB0EF11C8F019F
:1058B0003F01470140E1C42ED12CBE016D5B7F4FFB
:1058C000C6010E94D92A2596AEACBFAC2597D4015B
:1058D000AD92BD924D01BE016F5F7F4FC6014496F0
:1058E0000E94D92AB1E0AB1AB10849815A81E8E097
:1058F000AE16B10438F481E09A01245C3F4F293799
:10590000310508F080E0D3014D935D933D01811195
:105910005AC084E00E94A22B91E0811101C090E066
:105920009093372888E00E94A22B90E08093552A1C
:105930009093562A8AE00E94A22B91E0811101C027
:1059400090E09093742A8EE00E94A22B90E08093C6
:1059500016299093172980916E2A90916F2A0E94A0
:10596000310980916C2A90916D2A0E943109E09151
:105970006C2AF0916D2A808580FDFEC140EF50E0D9
:1059800062E070E08AE090E00E94CD1A87EF9FEE1F
:105990000E94801F80916E2A90916F2ADC011896D8
:1059A0002C9120FF07C0E0916C2AF0916D2A208590
:1059B00020FD29C00E94310980916C2A90916D2AA6
:1059C0000E943109E7CFE2E0CE0ED11CF0E2CF1603
:1059D000D10409F072CFA1E2B8E241E85AE2C7016E
:1059E0004096F701219131917F012D933D93F8016C
:1059F000219131918F01FA0121933193AF018E15DD
:105A00009F0579F786CF8091B8ED9091B9EDA0917F
:105A1000BAEDB091BBED2B968CAF9DAFAEAFBFAFE3
:105A20002B972091372881E0282730E042E050E092
:105A3000BE01695B7F4F85E090EF0E94D51F21E09A
:105A4000892B09F020E02093372867E378E284E08F
:105A500090E00E94C22A8091BCED9091BDEDA09192
:105A6000BEEDB091BFED27968CAF9DAFAEAFBFAF8F
:105A700027972091152930E042E050E0BE016D5B90
:105A80007F4F82E190EF0E94D51F21E0019709F03E
:105A900020E02093152965E179E286E090E00E94FC
:105AA000C22A2091742A81E0282730E042E050E0A9
:105AB000BE01695B7F4F8AE190EF0E94D51F21E014
:105AC000892B09F020E02093742A64E77AE28AE0C7
:105AD00090E00E94C22A2091152881E0282730E01A
:105AE00042E050E0BE01695B7F4F86E290EF0E948A
:105AF000D51F21E0892B09F020E02093152865E1CE
:105B000078E28CE090E00E94C22A20911629309120
:105B1000172943E050E06BE078E282E390EF0E94C7
:105B2000D51F809316299093172966E179E28EE0BC
:105B300090E00E94ED2A809116299091172963E048
:105B400070E00E945655FC01EE0FFF1FEE5DF14123
:105B5000808180930A2882E2E0ECFDEEDE0111965E
:105B600001900D928A95E1F72091552A3091562A9D
:105B700041E150E0BE016F5F7F4F88E390EF0E94EC
:105B8000D51F8093552A9093562A65E57AE288E0DE
:105B900090E00E94ED2A80E00E94D22BBE016D5B56
:105BA0007F4F90E080E00E94D92A25968EAD9FAD70
:105BB00025971816190624F480930828909309282D
:105BC000BE016F5F7F4F82E090E00E94D92A8981F9
:105BD0009A811816190624F48093062890930728B2
:105BE00087E190E00E94A855FC01209106283091A1
:105BF000072840910828509109288FEF9FEF83874D
:105C0000948785879687838B948B88E090E0858B3B
:105C1000968B40835183228333831086118682E0E2
:105C200090E08483958384E190E086839783E0937A
:105C3000BE2AF093BF2AE091722AF091732AF89459
:105C400017821086118612867894E091682AF09166
:105C5000692AF8941782108611861286789487E054
:105C600090E08093662A9093672A8091552A9091BC
:105C7000562A8093A72D9093A82D80E00E94A52BF3
:105C80001092C72D1092C82D04E510E00093C92D85
:105C90001093CA2D81E790EF0E94801F1092C72DAC
:105CA0001092C82D8FE690E08093C92D9093CA2D55
:105CB0008DE790EF0E94801F80E00E94AC228091CF
:105CC0003E2890913F280E94962284E890E080939D
:105CD000C72D9093C82D0093C92D1093CA2D88E02D
:105CE00090E00E94B3208FEF9FEF80934528909320
:105CF00046280E94D32FE0901A29F0901B2903E434
:105D000010E02CE330E046E350E064EB70E08BEB16
:105D10009DE20E94EB11E0901829F09019292CE3E4
:105D200030E046E350E064EB70E08BEB9DE20E94D4
:105D3000A517E0901829F090192901E410E02AE352
:105D400030E047E350E065EB70E08BEB9DE20E94B2
:105D5000A517C65BDF4FCDBFDEBFDF91CF911F918F
:105D60000F91FF90EF90DF90CF90BF90AF909F90FA
:105D70008F907F906F900895E0916E2AF0916F2A36
:105D8000808580FD0BCF40EF50E061E070E090E057
:105D900080E00E94CD1A81E490EF0E94801F8091E4
:105DA0006E2A90916F2AFC01208520FF07C0E091A8
:105DB0006C2AF0916D2A208520FD09C00E943109CE
:105DC00080916C2A90916D2A0E943109E8CF10923F
:105DD000C72D1092C82D89E3E82EF12CE092C92D31
:105DE000F092CA2D8BE490EF0E94801F60ED77E067
:105DF00080E090E00E94BA0784E10E9469070FEFFB
:105E000013E09801281B390B25962EAF3FAF25973D
:105E100098E7C92ED12CC092C72DD092C82DE09200
:105E2000C92DF092CA2D83E590EF0E94801F259620
:105E30008EAD9FAD25970E94B32088E590EF0E941C
:105E4000801F68EE73E080E090E00E94BA07109235
:105E5000C72D1092C82D24E5E22EF12CE092C92D19
:105E6000F092CA2D8AE590EF0E94801F60ED77E0E6
:105E700080E090E00E94BA0784E10E946907D8019F
:105E8000A81BB90BCD01A983BA83C092C72DD092AC
:105E9000C82DE092C92DF092CA2D0E94B3202596FC
:105EA0008EAD9FAD25978D599F4F29813A818217DD
:105EB0009307DCF084E10E946907F801E81BF90B05
:105EC000E983FA8344E650E063E070E088E790E01D
:105ED0000E94CD1A89819A810E94B32064E670E005
:105EE00080E090E00E94BA07DACF88E790E08093E4
:105EF000C72D9093C82D8FE690E08093C92D909385
:105F0000CA2D82E690EF0E94801F1092C72D10923A
:105F1000C82D8AE890E08093C92D9093CA2D2596CC
:105F20008EAD9FAD259784389340C4F589819A81C1
:105F3000883E93409CF585E690EF0E94801F259651
:105F40008EAD9FAD2597809308289093092889816D
:105F50009A81809306289093072868E078E290E081
:105F600080E00E94ED2A66E078E282E090E00E9404
:105F7000ED2A68EB7BE080E090E00E94BA07F12C0C
:105F8000E12C07E810E020EF30E04CE150E070E059
:105F900060E08BEB9DE20E94EB1100CE8AE690EF71
:105FA0000E94801FE6CFEF92FF920F931F938FE026
:105FB0000E946907893E23E0920774F4833523E049
:105FC00092070CF077C0853691050CF076C01F91D2
:105FD0000F91FF90EF90089581E090E02091452887
:105FE000309146282817390791F3809345289093DC
:105FF000462860E087E00E94C72370E060E080E10F
:106000000E948406F12CE12C0BE110E028E730E03F
:106010004CE650E06CE370E08BEB9DE20E94EB11EC
:1060200088E790E08093C72D9093C82D8FE690E08D
:106030008093C92D9093CA2D809145289091462830
:106040008130910509F45AC0D8F1029709F45BC078
:106050000E94F71A8091452890914628892B61F07B
:106060008091E42A882349F02091452830914628E0
:1060700081E02130310509F080E08093E32A8091AE
:106080003728882309F4A3CF0E94EA076093BA2A2D
:106090007093BB2A8093BC2A9093BD2A8091B92A21
:1060A000882309F494CF80E01F910F91FF90EF9027
:1060B0000C94D22B82E090E091CF90E080E08ECFE4
:1060C00080EB90EF0E94801F6091472870914828D4
:1060D0008091492890914A280E9425522091312888
:1060E0003091322840913328509134280E947B51BE
:1060F0000E94ED5141E00E945020AACF85EB90EF25
:106100000E94801FA5CF8AEB90EFFACF4F925F924B
:106110006F927F928F929F92AF92BF92CF92DF92B7
:10612000EF92FF920F931F93CF93DF93CDB7DEB71C
:106130002E97CDBFDEBF80914528909146280197CC
:1061400009F088C182E00E94440721E030E0892BF9
:1061500011F030E020E02093D52A3093D62A82E057
:106160000E944407019709F475C12091E32A29830D
:1061700081E082278093D12A0E948B074B015C012A
:106180003981332309F42EC180910D2990910E2974
:10619000A0910F29B0911029A5019401281B390B5A
:1061A0004A0B5B0BCA01B9010E94235269837A83AF
:1061B0008B839C8320E030E044EB52E40E947B51CF
:1061C00020E030E040E05FE30E940A510E94ED5180
:1061D0006B01770FEE08FF080091442C1091452CBD
:1061E000D8018C918E7F8C938C918670823009F4CB
:1061F0005FC0843051F081110FC044E0CC0CDD1C35
:10620000EE1CFF1C4A95D1F707C062E0F694E794B4
:10621000D794C7946A95D1F780E090E0A1E0B0E010
:106220008093522C9093532CA093542CB093552CC4
:106230009701442755272B873C874D875E872093FE
:10624000462C3093472C4093482C5093492CC7013F
:10625000B6018827992760934A2C70934B2C809322
:106260004C2C90934D2C232B242B252B09F444C02C
:10627000412C512C32016394A30192012150310928
:10628000410951092D833E834F8358876130710541
:1062900081059105A9F4C701B6010E94D8502B874A
:1062A0003C874D875E874D805E806F807884E4CF29
:1062B00053E0CC0CDD1CEE1CFF1C5A95D1F7ACCF83
:1062C00060934A2C70934B2C80934C2C90934D2CC4
:1062D0004092522C5092532C6092542C7092552C18
:1062E0002B853C854D855E852093462C3093472C2D
:1062F0004093482C5093492C8091522C9091532CD0
:10630000A091542CB091552C0197A109B10980930B
:10631000522C9093532CA093542CB093552C409115
:106320004A2C50914B2C60914C2C70914D2C411566
:1063300051056105710561F041505109610971090B
:1063400040934A2C50934B2C60934C2C70934D2CC3
:106350004091462C5091472C6091482C7091492CCB
:1063600040934E2C50934F2C6093502C7093512C93
:10637000452B462B472B21F480914A2C90914B2C96
:10638000D8011C968D939C931D971A961D921C9272
:106390001B978C9181608C93C501B4010E9423529C
:1063A0006B017C0120E030E040EC5FE369817A81A1
:1063B0008B819C810E9432539B01AC01C701B601C5
:1063C0000E940A5120E030E04AE754E40E947B51E9
:1063D0000E94F4516093DF2A7093E02A8093E12AAF
:1063E0009093E22A80920D2990920E29A0920F2973
:1063F000B09210298091C02A811104C08091D12AC5
:10640000882341F180913728882321F10E94EA07EF
:106410006093BA2A7093BB2A8093BC2A9093BD2ABA
:106420008091B92A8823B1F080E02E96CDBFDEBFDF
:10643000DF91CF911F910F91FF90EF90DF90CF9060
:10644000BF90AF909F908F907F906F905F904F9094
:106450000C94D22B2E96CDBFDEBFDF91CF911F9132
:106460000F91FF90EF90DF90CF90BF90AF909F90F3
:106470008F907F906F905F904F9008950E94EA07F1
:106480006093B52A7093B62A8093B72A9093B82A5E
:106490008091972A9091982A63E070E00E94565567
:1064A000892B01F564EF71E080E090E00E94BA076B
:1064B00070E060E08BEB9DE20E947C1864EF71E07D
:1064C00080E090E00E94BA070E94ED4F23E030E0A8
:1064D00040E050E00E9475506E5F7F4F6093192836
:1064E00070931A280E94ED4F23E030E040E050E026
:1064F0000E9475506093A72A7093A82A0E94ED4FBE
:1065000022E330E040E050E00E947550FB014091F2
:10651000992A50919A2A4115510509F47CC04330BB
:10652000510509F478C02091C32D3091C42D261B4C
:10653000370B20939B2A30939C2A4230510534F02C
:10654000E091C52DF091C62DE61BF70BE0939D2A37
:10655000F0939E2A2091C32D3091C42D42305105D5
:1065600014F430E020E02093A52A3093A62A4115A8
:10657000510529F030E020E04330510521F420910D
:10658000C52D3091C62D2093A12A3093A22A2091A7
:10659000C32D3091C42D4230510514F030E020E07D
:1065A0002093A32A3093A42A4115510539F0433092
:1065B000510599F14091C52D5091C62D40939F2AC8
:1065C0005093A02A0E94ED4F2DE730E040E050E0CC
:1065D0000E947550675E7F4F8F4F9F4F0E942552DC
:1065E00020E030E048E452E40E947B5160931D2893
:1065F00070931E2880931F28909320280E94ED4FAF
:106600002FEF3FEF40E050E00E94755060931B2851
:1066100070931C2808959B018CCF50E040E0CECFB2
:106620003F924F925F926F927F928F929F92AF9222
:10663000BF92CF92DF92EF92FF920F931F93CF936F
:10664000DF93CDB7DEB72A97CDBFDEBF8091452857
:1066500090914628029709F0F6C2809111299091F5
:1066600012290196809311299093122980910B2968
:1066700090910C29019680930B2990930C292091DD
:10668000092930910A292F5F3F4F29873A872093A4
:10669000092930930A290E948B076B017C018090A5
:1066A0000D2990900E29A0900F29B09010298114E7
:1066B0009104A104B10409F4BDC08C149D04AE047E
:1066C000BF0408F0B7C04090382850903928609037
:1066D0003A2870903B2860910A2870E090E080E0B2
:1066E0000E94255220913128309132284091332840
:1066F000509134280E9432539B01AC0160E070E657
:106700008AE697E40E947B5169837A838B839C831A
:10671000C701B6010E9423526D837E838F839887C1
:10672000C501B4010E9423529B01AC016D817E81A1
:106730008F8198850E9409519B01AC0169817A8102
:106740008B819C810E947B5120E030E04AE754E439
:106750000E9432534B015C018091072990910829D6
:10676000FC01EE0FFF1FEE0FFF1FE552F74D808279
:106770009182A282B38201966BE070E00E9456552E
:10678000809307299093082989859A850B971CF196
:106790008CE2EBEDF8E2AFEAB8E201900D928A9557
:1067A000E1F72DEB3AE144E050E06BE070E08FEA76
:1067B00098E20E94D84D8091C3289091C428A0915E
:1067C000C528B091C6288093382890933928A09383
:1067D0003A28B0933B28A301920160913828709128
:1067E000392880913A2890913B280E9409510E94B3
:1067F000ED519B0177FF04C022273327261B370B5F
:10680000B901330F880B990B0E942552A301920105
:106810000E947B5120E030E040E85EE30E942D536F
:10682000181644F48092382890923928A0923A2879
:10683000B0923B28C0920D29D0920E29E0920F29E8
:10684000F0921029409038285090392860903A28CA
:1068500070903B28B301A2018AEC9CE20E94F31CD9
:106860000E94EF5369837A838B839C8300910A286B
:1068700010E0B801012E000C880B990B0E942552E4
:106880006B017C01209131283091322840913328CE
:10689000509134280E9432530E94EF530E94ED51D0
:1068A0006D837E832091E42A222319F13090572AA8
:1068B000072E000C880B990B0E9425524B015C019E
:1068C0008D819E8163E070E00E945655072E000C7A
:1068D000880B990B0E9425529B01AC01C501B401A4
:1068E000332009F49CC00E940A510E94ED516D832F
:1068F0007E838091112990911229ED81FE818E175E
:106900009F0709F0B5C18091572A91E089278093AC
:10691000572A10921129109212298091AE288823AB
:1069200009F44BC180910B2990910C29B8010E9468
:106930005655892B09F041C11092AE2810920B29AF
:1069400010920C298090AA289090AB28A090AC2897
:10695000B090AD288092312890923228A0923328AE
:10696000B09234288091452890914628029709F0EA
:1069700059C0A7019601C301B2010E94325320E021
:1069800030E040EC51E40E947B510E94EF530E94A2
:10699000ED5140E00E9450206091472870914828B6
:1069A0008091492890914A280E9425529B01AC0170
:1069B00060EC71EE84E69CE40E947B5120913128CA
:1069C0003091322840913328509134280E9432531C
:1069D00020E030E044EB52E40E947B510E94EF53F0
:1069E0000E94F4516B017C012091442C3091452C84
:1069F0002D833E83F90180818E7F80838081867024
:106A0000823009F46DC0843019F1811128C0A4E0EE
:106A1000CC0CDD1CEE1CFF1CAA95D1F720C00E94F7
:106A2000095163CF8091452890914628892B09F020
:106A3000B3CF609147287091482880914928909160
:106A40004A280E942552A50194010E947B519FCFA4
:106A500012E0F694E794D794C7941A95D1F780E0A2
:106A600090E0A1E0B0E08093522C9093532CA0933F
:106A7000542CB093552C9701442755272093462C2E
:106A80003093472C4093482C5093492CC701B601B2
:106A90008827992760934A2C70934B2C80934C2C19
:106AA00090934D2C2115310541055105C9F1412C1B
:106AB000512C3201639453014201F1E08F1A910885
:106AC000A108B108613071058105910589F4C701FC
:106AD000B601A50194010E94D85024013501EBCFE5
:106AE000B3E0CC0CDD1CEE1CFF1CBA95D1F7B7CF80
:106AF00060934A2C70934B2C80934C2C90934D2C8C
:106B00004092522C5092532C6092542C7092552CDF
:106B10002093462C3093472C4093482C5093492C7B
:106B20008091522C9091532CA091542CB091552CC3
:106B30000197A109B1098093522C9093532CA093F3
:106B4000542CB093552C40914A2C50914B2C609171
:106B50004C2C70914D2C411551056105710561F06A
:106B6000415051096109710940934A2C50934B2CB3
:106B700060934C2C70934D2C4091462C5091472C97
:106B80006091482C7091492C40934E2C50934F2C7F
:106B90006093502C7093512C452B462B472B21F49E
:106BA00080914A2C90914B2CED81FE8184879587B2
:106BB0001286138680818160808380910D29909157
:106BC0000E29A0910F29B0911029892B8A2B8B2B8C
:106BD00079F169817A818B819C810E94ED516B01F1
:106BE0007C018091CF2A9091D02A092E000CAA0B0B
:106BF000BB0BC816D906EA06FB06D1F0A0910A28FD
:106C0000B0E0A70196010E94945028E130E040E0F6
:106C100050E00E947550CA01B9010E9425520E949D
:106C2000ED5140E00E945020C092CF2AD092D02A4D
:106C300080914B2881110E94141B81E090E0809389
:106C4000D52A9093D62A2A96CDBFDEBFDF91CF9169
:106C50001F910F91FF90EF90DF90CF90BF90AF907A
:106C60009F908F907F906F905F904F903F9008958E
:106C70002D813E8137FF04C02F5F3F4F2D833E8320
:106C8000ED81FE81F595E795E817F907E4F6109296
:106C9000D52A1092D62AD7CF1F920F920FB60F92F5
:106CA00011242F933F934F935F936F937F938F9311
:106CB0009F93AF93BF93EF93FF9385E00E94BC0532
:106CC000FF91EF91BF91AF919F918F917F916F91C4
:106CD0005F914F913F912F910F900FBE0F901F909A
:106CE00018951F920F920FB60F9211242F933F9376
:106CF0004F935F936F937F938F939F93AF93BF93C4
:106D0000EF93FF9384E00E94BC05FF91EF91BF9148
:106D1000AF919F918F917F916F915F914F913F9133
:106D20002F910F900FBE0F901F9018951F920F92EA
:106D30000FB60F9211242F933F934F935F936F934E
:106D40007F938F939F93AF93BF93EF93FF9383E0D2
:106D50000E94BC05FF91EF91BF91AF919F918F91E0
:106D60007F916F915F914F913F912F910F900FBE47
:106D70000F901F9018951F920F920FB60F9211242B
:106D80002F933F934F935F936F937F938F939F9333
:106D9000AF93BF93EF93FF9382E00E94BC05FF91F6
:106DA000EF91BF91AF919F918F917F916F915F9183
:106DB0004F913F912F910F900FBE0F901F901895FC
:106DC0001F920F920FB60F9211242F933F934F9360
:106DD0005F936F937F938F939F93AF93BF93EF9343
:106DE000FF9381E00E94BC05FF91EF91BF91AF91AD
:106DF0009F918F917F916F915F914F913F912F91D3
:106E00000F900FBE0F901F9018951F920F920FB604
:106E10000F9211242F933F934F935F936F937F9320
:106E20008F939F93AF93BF93EF93FF9380E00E9464
:106E3000BC05FF91EF91BF91AF919F918F917F9191
:106E40006F915F914F913F912F910F900FBE0F90D7
:106E50001F9018951F920F920FB60F9211242F9327
:106E60003F934F935F936F937F938F939F93AF93D2
:106E7000BF93EF93FF9380E09DE20E94D704FF91C0
:106E8000EF91BF91AF919F918F917F916F915F91A2
:106E90004F913F912F910F900FBE0F901F9018951B
:106EA0001F920F920FB60F9211242F933F934F937F
:106EB0005F936F937F938F939F93AF93BF93EF9362
:106EC000FF9380E09DE20E94F505FF91EF91BF9155
:106ED000AF919F918F917F916F915F914F913F9172
:106EE0002F910F900FBE0F901F9018951F920F9229
:106EF0000FB60F9211242F933F934F935F936F938D
:106F00007F938F939F93AF93BF93EF93FF9389EA00
:106F10009BE20E94D704FF91EF91BF91AF919F91A7
:106F20008F917F916F915F914F913F912F910F9032
:106F30000FBE0F901F9018951F920F920FB60F92D1
:106F400011242F933F934F935F936F937F938F936E
:106F50009F93AF93BF93EF93FF9389EA9BE20E94C5
:106F6000F505FF91EF91BF91AF919F918F917F9127
:106F70006F915F914F913F912F910F900FBE0F90A6
:106F80001F9018951F920F920FB60F9211242F93F6
:106F90003F934F935F936F937F938F939F93AF93A1
:106FA000BF934091452A5091462A6091472A70919B
:106FB000482A8091432A9091442A20914F2A309167
:106FC000502A420F531F611D711D20914D2A30918F
:106FD0004E2A820F931F883E23E0920730F0885E8E
:106FE00093404F5F5F4F6F4F7F4F8093432A909343
:106FF000442A4093452A5093462A6093472A709327
:10700000482A8091492A90914A2AA0914B2AB0910E
:107010004C2A0196A11DB11D8093492A90934A2ABA
:10702000A0934B2AB0934C2A81E08093B60ABF917B
:10703000AF919F918F917F916F915F914F913F9110
:107040002F910F900FBE0F901F9018951F920F92C7
:107050000FB60F9211242F933F934F935F936F932B
:107060007F938F939F93AF93BF93EF93FF93809101
:107070004E2C90914F2CA091502CB091512C0197F7
:10708000A109B10980934E2C90934F2CA093502CC2
:10709000B093512C181619061A061B063CF1892BC1
:1070A0008A2B8B2BB9F18091462C9091472CA09183
:1070B000482CB091492C0097A105B10591F080931F
:1070C0004E2C90934F2CA093502CB093512CE091C8
:1070D000442CF091452C8091522C9091532C848714
:1070E0009587E091562CF091572C099581E080937B
:1070F000A60AFF91EF91BF91AF919F918F917F91E0
:107100006F915F914F913F912F910F900FBE0F9014
:107110001F90189540914A2C50914B2C60914C2C0B
:1071200070914D2C4115510561057105A9F0E09153
:10713000442CF091452C4487558782859385B0E097
:10714000A0E084179507A607B70784F28091522C18
:107150009091532C848795878091462C9091472C51
:10716000A091482CB091492C80934E2C90934F2C99
:10717000A093502CB093512CB4CF1F920F920FB606
:107180000F9211242F933F934F935F936F937F93AD
:107190008F939F93AF93BF93CF93EF93FF93C09140
:1071A000AB08C2FF0AC01092362A1092352A1092FC
:1071B000342A84E00E94CB0B14C0C6FF2FC08091FC
:1071C000332A813051F48091362AE091312AF091AE
:1071D000322A90E009951092332AC0FF14C00E9411
:1071E000DB0BFF91EF91CF91BF91AF919F918F9169
:1071F0007F916F915F914F913F912F910F900FBEB3
:107200000F901F90189580E48093AB0881E00E9456
:10721000CB0B8091AB0885FFE4CFE1CFC7FF5CC00B
:10722000C3FF08C01092362A1092352A1092342AD1
:1072300083E0C0CF8091A90880668093A9088091DF
:10724000AB0881FF2CC08091352A882349F08091BA
:10725000AB0884FF05C082E08093AA0881E0AACF32
:107260009091352A8091342A9817A8F4E091352A14
:1072700080912C2A90912D2AE80FF92FF11D808101
:107280008093AD088091352A8F5F8093352A83E003
:107290008093AA08A6CF82E08093AA088BCF909112
:1072A000362A8091302A981790F48091AD08E091A9
:1072B000362A20912E2A30912F2AE20FF32FF11D2A
:1072C00080838091362A8F5F8093362AE0CF86E0D4
:1072D0008093AA0882E06ECF85E06CCF1F920F9258
:1072E0000FB60F9211242F933F938F939F93EF9399
:1072F000FF938091A508982F9C70E1F08091A508DC
:1073000094E082FF93E09093412A8093A50881E066
:1073100090E08093372A9093382A1092422AFF9166
:10732000EF919F918F913F912F910F900FBE0F90F2
:107330001F90189586FF4EC020913E2A90913D2ABD
:107340008091A50884FF15C080913A2A882379F09E
:1073500083E08093A40885E08093412A1092422A1A
:1073600081E090E08093372A9093382AD8CF81E04B
:10737000F0CF80913C2A821790F4E0913C2A8091D2
:107380003F2A9091402AE80FF92FF11D80818093C8
:10739000A80880913C2A8F5F80933C2AC0CF8091BF
:1073A0003B2A891760F484E090E08093372A909319
:1073B000382A8091392A81608093A708B0CF8091C4
:1073C0003A2A882329F083E08093A40881E0C4CF7F
:1073D00081E0FACF87FF40C090913B2A80913D2AFF
:1073E0009817D8F48091A808E0913B2A20912A2A86
:1073F00030912B2AE20FF32FF11D808380913B2ADD
:107400008F5F80933B2A90913D2A80913B2A891778
:10741000D8F482E08093A40882CF80913A2A88230E
:1074200089F087E08093A40882E08093412A10923B
:10743000422A81E090E08093372A9093382A109274
:107440003D2A6DCF85E0EECF80913A2A882311F056
:1074500087E0BACF85E0B8CF86E07ECFEF92FF928B
:107460000F931F93CF93DF93A0E0BDE212961D927E
:107470001C92139748EE53E060E070E014964D9331
:107480005D936D937C93179726EC3EEE2D933C9382
:10749000119780E298E01C968D939C931D971E9601
:1074A0001C921E9781E01F968C931F9794E0509634
:1074B0009C93509752961C92529753961C925397B6
:1074C00054961C92549755961C9255979BE156964C
:1074D0009C93569757961C92579758961C9258977C
:1074E0001092992D10929A2DE9EAFBE212821382F2
:1074F00044835583668377832083318320E638E095
:107500002487358798E1968799E1978790E4908B57
:10751000128A138A148A158A96E2968B178A108E1D
:107520001092422C1092432CE4E4FCE220E83AE072
:107530002083318312821382148215820AE010E0C4
:1075400020E030E006831783208731871286138678
:10755000148615860FEF1FEF20E030E006871787AF
:10756000208B318BECE5FCE200E019E02DE330E00C
:1075700000831183228333831482158221E030E05B
:1075800026833783C0E7DCE2E0EEFEEEE883F98392
:107590001F8212E01E839CE09A839DE09C839BE007
:1075A0009B8398E09D83E4E6FCE21282138244838D
:1075B0005583668377834EEF5EEE40835183EBEB1A
:1075C000FDE21282138260EF70E06483758340E411
:1075D00051E0468357836087718742875387168AB5
:1075E0001486158616861786858B848B4FEF5FEF82
:1075F000428B538B408B518B878B108E118E128E4A
:1076000015AA89E086AB8AE087AB90AF11AE12AEC7
:1076100013AE14AE15AE16AE1092FA2D1092FB2DCD
:107620001092FC2D1092FD2DC78FD0A344E854E09A
:10763000458F568F93AB84E294E0838F948F11AB88
:107640008DEF82AB87EF84AB1092FE2D1092FF2D51
:107650001092002E8AE59FEE808391831092012E76
:107660001092022EE7EBFDE210821182EBE9FDE2BF
:107670008AE89FEE80839183A283B383148215826C
:1076800016821782248735870E94EA076093FC2CB4
:107690007093FD2C8093FE2C9093FF2C0E94EA07A0
:1076A000C9EEDCE2188219821A821B821C821D82BA
:1076B0001E821F82188619861A860E94EA076B8727
:1076C0007C878D879E878CE2E82EFF24F394EF86DB
:1076D000F88A04E110E0098B1A8BC6EDDCE218820F
:1076E00019821A821B821C821D821E821F821886AA
:1076F00019861A860E94EA076B877C878D879E878A
:10770000EF86F88A098B1A8BEAECFCE28AE999E9A0
:10771000A9E1BEE380839183A283B38380E090E0FC
:10772000A0EFB2E484839583A683B783EEEBFCE2FB
:107730004DEC5CEC6CE47DE34083518362837383A6
:1077400040E050E060E074E44483558366837783CF
:10775000E2EBFCE24AE959E969E97EE340835183BF
:107760006283738384839583A683B783DF91CF91EC
:107770001F910F91FF90EF900895CF93DF93CDB7B6
:10778000DEB7EA97CDBFDEBF88ED90E084BF90936F
:10779000610080E094E2A4EFB0E080931128909320
:1077A0001228A0931328B0931428809102068660B3
:1077B000809302068091000681608093000680918C
:1077C00002068F7C809302068091A0008F788093C0
:1077D000A000809102068061809302061092E2056B
:1077E00081E08093E40583E08093010A8FEF90E0CD
:1077F0008093260A9093270A80E890E08093380AC5
:107800009093390A80933A0A90933B0A80933C0AFA
:1078100090933D0A8BE08093000A8091E50581609A
:107820008093E5058091E50582608093E505E0E8B9
:10783000FAE037E02FEF90E885E0318324879587E1
:1078400080837096E03C0AE0F007B9F780E094E0AE
:107850008093532A9093542A8091532A9091542ACA
:107860002FEF30E0B9010E9461506093512A70936C
:10787000522A8091532A9091542AE8EEF3E0BF01F6
:107880000E94615060934F2A7093502A8091532A2E
:107890009091542ABF010E94615080934D2A909389
:1078A0004E2A2093BC0A3093BD0A8091B50A8160AC
:1078B0008093B50A84E08093B00A8091B00A816019
:1078C0008093B00A78941092002E40E050E0BA0104
:1078D0008BEB9DE20E94FD2888E28093022E80932C
:1078E000FF2D85E38093FE2D84E38093012E87E8AE
:1078F00090E08093032E9093042E80EF90E080938D
:10790000052E9093062EE8EEF7E09490E9EEF7E06E
:107910009A941FEF911609F47EC014915F0122E042
:10792000A20EB11C31968490082D0F778BEB9DE24F
:107930000E94CB0F8091F22D87FD09C0E091D62DDA
:10794000F091D72D80819091ED2D89238083E09156
:10795000D82DF091D92D80819091EF2D89238083AE
:10796000612F8BEB9DE20E94190FE091D82DF091D1
:10797000D92D80819091EE2D892B8083F501D12C1A
:10798000C12C10E0C016D106FCF48091F02D7F01CF
:10799000823089F48091EB2D882369F0DF016D91AD
:1079A0007D917D018BEB9DE20E94D40EEFEFCE1A0C
:1079B000DE0AF701E7CFBFEFEB1AFB0A64918BEB0E
:1079C0009DE20E94190FF2CF8091F22D87FD09C030
:1079D000E091D62DF091D72D80819091EC2D892BBF
:1079E00080838BEB9DE20E94BA0FF501E00FF11F3F
:1079F00087FE8ECF7F010FEFE01AF00A649170E0EE
:107A00006F3F710511F464EF71E090E080E00E9437
:107A1000BA07F7017DCF60E08BEB9DE20E946B100F
:107A200070E060E08BEB9DE20E947C1882E0809326
:107A3000CF2D8093D02D8CE00E94A22B91E081115C
:107A400001C090E09093152863E0811101C061E0CE
:107A50008BEB9DE20E946B1081E00E94A52B62E0FF
:107A600070E08FE00E941C0662E070E084E00E94FB
:107A70001C0662E070E085E00E941C068CE090E04D
:107A80000E94A8558C0145E064E00E94A21E00936C
:107A9000722A1093732A62E070E086E00E941C064E
:107AA00082E190E00E94A855FC01128213821482A8
:107AB0001582BAE0AB2EB12CA682B782108616E6EC
:107AC000C12E1EEED12EC082D18280936E2A909359
:107AD0006F2A86E0818BCF010E949A09E0916E2A7D
:107AE000F0916F2A02E3E02EF12CE682F78262E049
:107AF00070E087E00E941C0662E070E08CE00E946B
:107B00001C068CE090E00E94A8558C014CE067E0D8
:107B10000E94A21E0093682A1093692A62E070E016
:107B20008EE00E941C0682E190E00E94A855FC01B4
:107B30001282138214821582A682B7821086C082B6
:107B4000D18280936C2A90936D2A8EE0818BCF0135
:107B50000E949A09E0916C2AF0916D2AE682F782E0
:107B60008091B92D9091BA2D0E94445686E090E004
:107B70000E94A8558C0180E2D8018C9384E69CE297
:107B800011968D939C93129713961C92139780E2F3
:107B900090E014968D939C9315970093B92D1093B4
:107BA000BA2D84E69CE20E94B70D99249394F801C3
:107BB0009382C8010E94EE0D61E086E00E94952349
:107BC00061E085E00E94952361E084E00E949523B6
:107BD00061E087E00E94952362E082E00E949523A5
:107BE00062E080E00E94952361E083E00E9495239B
:107BF00061E081E00E94952382E190E00E94A85517
:107C0000FC011282138214821582A682B78210862A
:107C1000C082D1828093612A9093622A8FE0818B07
:107C2000CF010E949A09E091612AF091622AE682CE
:107C3000F78260914B28692584E00E94C72360E0A9
:107C400087E00E94C72361E083E00E94C72361E0D0
:107C500081E00E94C72360E086E00E94C72360E0C5
:107C600085E00E94C7231092B02A61E070E080E1B5
:107C70000E941C0670E060E080E10E94840661E0E2
:107C800070E081E10E941C0670E060E081E10E94EA
:107C9000840662E070E082E00E941C0666E870E301
:107CA00082E00E94310462E070E083E00E941C06E2
:107CB00080EA9AE08093442C9093452C8091A00A0E
:107CC0008E7F8093A00A9092A60A1092A10A84E067
:107CD0008093A00A80E090E0A4E0B0E08093582C6C
:107CE0009093592CA0935A2CB0935B2C8091A00AAE
:107CF0008E7F8093A00A8091A00A8670F0E48F2E78
:107D0000F2E49F2EFFE0AF2EB12C853070F490E0AE
:107D1000FC01EE0FFF1FE80FF91FE758F1418081CA
:107D20009181A2814C01AA2EB12C9501442755279F
:107D3000C501B40188279927C12CD12C7601E39481
:107D4000F1E0CF1AD108E108F10861307105810531
:107D5000910539F4C501B401A70196010E94D850DC
:107D6000EFCF60934A2C70934B2C80934C2C9093C4
:107D70004D2C2093462C3093472C4093482C509305
:107D8000492CC092522CD092532CE092542CF09259
:107D9000552C611571058105910561F061507109DE
:107DA0008109910960934A2C70934B2C80934C2C41
:107DB00090934D2C20934E2C30934F2C4093502C6D
:107DC0005093512C232B242B252B21F4C0904A2C8B
:107DD000D0904B2CC092AC0AD092AD0A1092AA0A55
:107DE0001092AB0A8091A00A81608093A00A83E977
:107DF0009CE18093562C9093572C81E08093A60AA7
:107E00008093A50A8091A00A8E7F8093A00A80911A
:107E1000A00A8670853008F04DC090E0FC01EE0F9E
:107E2000FF1FE80FF91FE659F141C080D180E280C1
:107E3000F12C80E090E0A1E0B0E08093522C909390
:107E4000532CA093542CB093552C970144275527BD
:107E50002093462C3093472C4093482C5093492C28
:107E6000C701B6018827992760934A2C70934B2C41
:107E700080934C2C90934D2C2115310541055105D3
:107E8000C9F1412C512C320163945301420101E0AC
:107E9000801A9108A108B10861307105810591052A
:107EA00089F4C701B601A50194010E94D8502401AC
:107EB0003501EBCF80E9C82E80EDD82E83E0E82E87
:107EC000F12CB7CF60934A2C70934B2C80934C2CA1
:107ED00090934D2C4092522C5092532C6092542CE3
:107EE0007092552C2093462C3093472C4093482C6D
:107EF0005093492C8091522C9091532CA091542C4A
:107F0000B091552C0197A109B1098093522C9093FF
:107F1000532CA093542CB093552C40914A2C509143
:107F20004B2C60914C2C70914D2C411551056105E5
:107F3000710561F0415051096109710940934A2C62
:107F400050934B2C60934C2C70934D2C4091462CAD
:107F50005091472C6091482C7091492C40934E2CA5
:107F600050934F2C6093502C7093512C452B462BE3
:107F7000472B21F480914A2C90914B2C8093AC0A92
:107F80009093AD0A1092AA0A1092AB0A8091A00AAF
:107F900081608093A00A83EA9AE18093A92D90934F
:107FA000AA2D1092AB2D1092AC2D80E193E380931B
:107FB000AF2D9093B02D89E89BE28093B12D9093E3
:107FC000B22D89E69BE28093B32D9093B42D84E784
:107FD0009BE28093B52D9093B62D8DE397E280932D
:107FE000AD2D9093AE2D0091552A1091562A809177
:107FF0009D2D90919E2DDC01ED91FC910684F785DD
:10800000E02D42E15AE760E070E0099510929F2D63
:108010001092A02D0093A72D1093A82D0E94EA077F
:108020006093BA2A7093BB2A8093BC2A9093BD2A8E
:10803000611571058105910511F00E943C508091F8
:10804000372881110E943E3281E00E94D22B0E948B
:10805000EA076093FC2C7093FD2C8093FE2C909388
:10806000FF2C80914528909146288091D52A9091A7
:10807000D62A2091D72A211109C021E0009709F0C2
:1080800020E02093D42A21E02093D72A2091D42ADB
:1080900028171906C1F061E0892B09F460E087E038
:1080A0000E94C72361E08091D52A9091D62A892B1E
:1080B00009F460E06093D42A80914B28882319F05A
:1080C00086E00E94C7238091D32A882309F48DC0BB
:1080D0001092D32A8091452890914628892B29F027
:1080E0008091E32A882309F46DC0209116283091ED
:1080F00017286091582A7091592A80915A2A909194
:108100005B2A032E000C440B550B0E94D850609341
:10811000582A7093592A80935A2A90935B2A809107
:10812000F02C9091F12C0197029708F053C0E09148
:108130004028F0914128CF010A9608E010E0B801EC
:108140000E9456559C01220F331F2F57354DCF01EA
:108150000996B8010E945655FC01EE0FFF1FEF571C
:10816000F54DD9018D919C9120813181821B930B1A
:10817000865A9F4F80931628909317288091E42A5F
:108180008823C1F08091572A22EE3FEF811102C06F
:108190002EE130E08091162890911728820F931FCE
:1081A00080931628909317288091572A91E0892769
:1081B0008093572A8091B22A882379F01092B22AAC
:1081C0000E94912780E090E0892B09F440CF0E9423
:1081D00000003DCF90E080E0CBCF80914B288823FA
:1081E00089F381E08093B32AEDCF8091D22A88234E
:1081F00019F00E942E28E6CF8091D12A882381F1A0
:108200000E942E28609138287091392880913A2850
:1082100090913B280E94EF530E94ED516B017C012D
:108220001C141D041E041F046CF68091CF2A90912B
:10823000D02A8C33910554F08C199D0997FF03C007
:1082400091958195910903970CF4BCCF40E0C7014B
:10825000B6010E945020C092CF2AD092D02AB2CF2D
:108260008091C72A81110DC00E94EA076093C32A3A
:108270007093C42A8093C52A9093C62A81E0809384
:10828000C72A4091C32A5091C42A6091C52A70918F
:10829000C62A4115510561057105E1F08091FC2C5C
:1082A0009091FD2CA091FE2CB091FF2C841B950B7E
:1082B000A60BB70B813D9740A105B10558F080E0B2
:1082C0000E94AC221092C32A1092C42A1092C52A8E
:1082D0001092C62A80919D2D90919E2DDC01ED91EA
:1082E000FC910084F185E02D0995181619060CF013
:1082F00074C080919D2D90919E2DDC01ED91FC919B
:108300000284F385E02D0995282F80919F2D90916F
:10831000A02D8130910509F49EC18230910509F4A8
:10832000AFC1892B09F059C088E0820F8530A0F1D8
:108330004091A72D5091A82D4115510541F0822F54
:108340008F7090E001964817590709F046C0822FB8
:10835000203F08F4807F8093A42D883FD1F1F0F472
:10836000803949F1803B91F180919D2D90919E2D16
:10837000DC01ED91FC910190F081E02D622F0995D7
:1083800080919D2D90919E2DDC01ED91FC910680B8
:10839000F781E02D099521C0822FDDCF8B3F09F4B5
:1083A00055C18C3F09F44DC18A3FF1F68BE99DE23E
:1083B0000E943D1A12C081E090E08093A12D90931D
:1083C000A22D80939F2D9093A02D07C081E090E077
:1083D000F8CF8BE99DE20E94451A0091612A109125
:1083E000622AF801808580FD15C00E94EA07D80145
:1083F0001996CD90DD90ED90FC901C976C197D093D
:108400008E099F0960935D2A70935E2A80935F2A8C
:108410009093602AC0905D2AD0905E2AE0905F2AF7
:10842000F090602AC8010E94310980915C2A811174
:1084300052C18091612A9091622A0E94290981117A
:1084400007C0B8ECCB16D104E104F1040CF443C12D
:1084500080913728882309F42FC10E94EA0760938E
:10846000BA2A7093BB2A8093BC2A9093BD2A80912C
:10847000B92A882309F420C180E00E94D22B809180
:10848000C12A9091C22A01968093C12A9093C22A50
:108490006BE070E00E945655892B99F483E00E94AE
:1084A00044079C0191E02115310509F090E080918D
:1084B0001828981731F090931828232B11F40E9454
:1084C000DD278091C12A9091C22A67E070E00E9466
:1084D0005655892BD1F58091722A9091732A0E946A
:1084E0008E1E6B01A090F02CB090F12CF2E0AF1A30
:1084F000B1086090DD2C7090DE2C02E0601A7108EB
:108500000091702A1091712A0617170709F4BDC14E
:10851000CB0181709927892B09F0B7C18091372849
:10852000882309F445C10E94EA076093BA2A709330
:10853000BB2A8093BC2A9093BD2A8091B92A8823B4
:1085400009F436C180E00E94D22B80914528909199
:108550004628892B09F0DBC38091C12A9091C22A59
:108560006DE070E00E9456558C01892B09F0CFC355
:108570008091792A811105C00E94EA0781E08093E9
:10858000792A85E10E9469071C0126E0221A310838
:1085900060E074E0681B790B072E000C880B990BC8
:1085A00036EF231633E0330608F490C30E942552B9
:1085B0006B017C01C092C22CD092C32CE092C42CDF
:1085C000F092C52CC092752AD092762AE092772A32
:1085D000F092782A8091742A882309F454C584E1A2
:1085E000E2EEFDEEDE01559601900D928A95E1F7DF
:1085F00084E1E6EFFDEEDE01119601900D928A9581
:10860000E1F720E030E040EA50E4C701B6010E9403
:10861000765187FD2EC520E030E44EE754E4C701D3
:10862000B6010E942D534E0149E1840E911C18168B
:108630000CF026C4A8E88A2EA3E19A2EA12CB12C16
:108640001DC58BE99DE20E94351AC7CE8BE99DE2DC
:108650000E942D1AC2CE8091A42D803939F0803B22
:1086600051F010929F2D1092A02DB7CE27FDF9CF7B
:108670002093A32D02C027FFFBCF82E090E0A1CE84
:108680008091A42D803971F0803B59F7E091AD2D98
:10869000F091AE2D309729F3422F6091A32D81E008
:1086A0000995DFCF27FDDDCF4091A32D61E08BE958
:1086B0009DE20E944D1AD5CF81E080935C2A809183
:1086C0004B288823F9F0E8ECCE16D104E104F1043C
:1086D000CCF40E94DD2780915C2A882309F4CFCE58
:1086E000E091612AF091622A808580FFC8CE1092C5
:1086F0005C2A10925D2A10925E2A10925F2A1092D4
:10870000602ABDCE11E060E081270E94332B80916A
:108710004B28882309F442C01092D52A1092D62AF9
:1087200060E087E00E94C723809145289091462809
:10873000892B59F5E091442CF091452C80818E7F56
:108740008083168380818E7F808316838091462C60
:108750009091472CA091482CB091492C80934E2C9D
:1087600090934F2CA093502CB093512C892B8A2B93
:108770008B2B79F08091522C9091532C8487958784
:108780001286138680818160808381E08093B22A83
:10879000A2CF80914A2C90914B2CF0CF209145286C
:1087A0003091462881E02130310581F380E0EECF21
:1087B000C601801B910B21E030E01816190614F059
:1087C0002FEF3FEF12E0A116B10408F0CDC0809169
:1087D000952A9091962A08964091932A5091942A2E
:1087E000841B950B68E070E00E945655AC01DC01DB
:1087F000AA0FBB1FFD01EF57F54D00811181F80154
:1088000017FF07C0EE27FF27E01BF10B31952195DD
:1088100031092130310549F4E531F1054CF4E830F6
:10882000F10544F52E0F3F1F0FC0E631F105FCF0B6
:10883000C901880F991F280F391F2E0F3F1F2F3195
:10884000310514F02EE130E017FF03C0319521957A
:108850003109AF57B54D2D933C9380914B28882318
:1088600061F0BA0181E090E00E94F6070AC0E930A9
:10887000F105C4F2220F331FD5CF61E080E00E94E2
:10888000DF20C092702AD092712A80916E2A909136
:108890006F2A0E94310980916C2A90916D2A0E9462
:1088A000310980916E2A90916F2A0E942909182F10
:1088B00080916C2A90916D2A0E942909982E11238B
:1088C000C9F080913728882371F00E94EA076093ED
:1088D000BA2A7093BB2A8093BC2A9093BD2A8091B8
:1088E000B92A81112FCE80916B2A882309F49BC06D
:1088F00010926B2A8091682A9091692A0E948E1E9C
:108900006B010091662A1091672A0617170709F470
:10891000FDC0CB0181709927892B09F0F7C08091A8
:108920003728882371F00E94EA076093BA2A70936F
:10893000BB2A8093BC2A9093BD2A8091B92A8111C9
:1089400001CEC601801B910B181619060CF0B2C09F
:1089500081E090E02091952A3091962A820F931F12
:1089600097FFABC00896FCCF42E06416710408F094
:1089700045C08091952A9091962A08964091932A15
:108980005091942A841B950B68E070E00E94565524
:10899000AC01FC01EE0FFF1FDF01AF5DB74D8D9104
:1089A0009C91280F391F29833A8381E090E08D8BB9
:1089B0009E8BDE0122303105D4F0119688E090E0E4
:1089C00089A79AA78D919C911197089714F0DE01C1
:1089D0009996EF5DF74D8D919C9180839183809165
:1089E0004B28882331F0BA0182E090E03DCF5596C4
:1089F000E5CF61E080E00E94792143CF8091E72AB2
:108A00009091E82A820F931F97FF02C00A96FCCF2D
:108A10006AE070E00E9456558093E72A9093E82A16
:108A20000E94921F2ECF52E0A516B104E0F480916F
:108A3000952A9091962A08962091932A3091942A0B
:108A4000821B930B68E070E00E945655FC01EE0F0C
:108A5000FF1FEF57F54D10821182AC0160E080E0FE
:108A60000E94DF2047CF82E068167104F0F4809105
:108A7000952A9091962A08962091932A3091942ACB
:108A8000821B930B68E070E00E945655FC01EE0FCC
:108A9000FF1FEF5DF74D21E030E020833183AC0113
:108AA00060E080E00E94792125CF10926A2A0E941E
:108AB000842620CF8FEF9FEF4DCF8770992780932B
:108AC000952A9093962AA2E0AA16B10408F08CC0C9
:108AD00008962091932A3091942A821B930B68E088
:108AE00070E00E94565520914B28222331F0BC01A2
:108AF00081E090E00E94F60705C0AC0161E080E0F3
:108B00000E94DF20C092662AD092672AE2E0AE1669
:108B1000B10408F44CC0F2E06F16710408F447C0C9
:108B20008091452890914628019709F440C0809192
:108B3000652A81113CC000916C2A10916D2AD801E0
:108B400018968C9180FD33C00E94EA07F8010185D8
:108B5000128523853485601B710B820B930B653F57
:108B600071408105910518F181E08093652A80911B
:108B7000632A9091642A0196833091050CF06BC0B2
:108B80008093632A9093642AE091632AF091642A87
:108B9000EE0FFF1FEE0FFF1FE857F141608171815B
:108BA000828193810E94ED51CB010E949F249920E4
:108BB00009F4CBCC80913728882371F00E94EA0712
:108BC0006093BA2A7093BB2A8093BC2A9093BD2AE3
:108BD0008091B92A8111B6CC8091652A882309F445
:108BE0003FC01092652AB1CCB2E06B167104C8F494
:108BF00008962091932A3091942A821B930B68E067
:108C000070E00E94565520914B28222321F0BC0190
:108C100082E090E06FCFAC0161E080E00E947921BA
:108C200071CF49E150E063E070E084E890E00E9499
:108C3000CD1A8091952A9091962A01960E94B32090
:108C40008FEF9FEF8093CD2D9093CE2D8093CB2DE2
:108C50009093CC2D57CF1092632A1092642A94CF10
:108C600002E0A016B10408F470CC12E061167104A1
:108C700008F46BCC8091952A9091962A019689836D
:108C80009A8321E030E02D8B3E8BFE010297E4F0C9
:108C9000319688E090E089A79AA780819181089712
:108CA00014F0FE01B9968081918120913E28309187
:108CB0003F288217930709F448CC80933E2890936D
:108CC0003F280E94962241CC7596E3CF0E94255200
:108CD000AB01BC018EEB9CE20E94F31C6B017C019A
:108CE0002091752A3091762A4091772A5091782ADE
:108CF0000E9409510E94ED519B0177FF04C0222779
:108D00003327261B370B233031050CF05BCC8091C9
:108D1000C12A9091C22A6BEB70E00E945655892BB4
:108D200011F40E94D32F2091C12A3091C22AC90187
:108D300065E270E00E945655892B09F084C349EE24
:108D40005CE266ED7CE282E090E00E943108182F40
:108D50008823C1F18091DD2C9091DE2C029702973F
:108D600088F58091DC2C882311F181E090E08093DC
:108D7000212890932228809323289093242880935D
:108D8000252890932628809327289093282880933D
:108D9000292890932A2880932B2890932C2880931D
:108DA0002D2890932E2880932F28909330288091FF
:108DB0004B28882309F494C26FEF7FEF82E090E0A4
:108DC0000E94F60746ED5CE269EE7CE290E080E00E
:108DD0000E943108882309F49FC68091F02C90915D
:108DE000F12C0297029778F58091EF2C882301F1FE
:108DF0001092812A1092822A1092832A1092842A39
:108E00001092852A1092862A1092872A1092882A18
:108E10001092892A10928A2A10928B2A10928C2AF8
:108E200010928D2A10928E2A10928F2A1092902AD8
:108E300080914B28882309F45AC26FEF7FEF81E0BD
:108E400090E00E94F60780913728882309F456C2E3
:108E50000E94EA076093BA2A7093BB2A8093BC2AC7
:108E60009093BD2A8091B92A882309F447C280E0F3
:108E70000E94D22BA7C985010430110509F48FC0C7
:108E800058015FEFA51AB50AF40181919191A19162
:108E9000B1914F018FA798ABA9ABBAABBC01CD0183
:108EA0000E942552A70196010E942D5318161CF707
:108EB000AA0CBB1CAA0CBB1CE1E0F0E0EC0FFD1FF0
:108EC000EA0DFB1D40805180628073805801AA0C1E
:108ED000BB1CAA0CBB1C88248394912C8C0E9D1E59
:108EE000A80CB91CD5016D917D918D919C910E942A
:108EF00025520E94ED516BA77CA78DA79EA7D50197
:108F000054960D911D912D913C9157970FAB18AF31
:108F100029AF3AAFC301B2010E9425520E94ED5120
:108F20004B015C010BA51CA52DA53EA5801A910A3D
:108F3000A20AB30A8BAA9CAAADAABEAAC701B6010F
:108F40000E94ED518FA898ACA9ACBAAC6819790908
:108F50008A099B092BA93CA94DA95EA90E943A55F3
:108F60002FA538A949A95AA9281939094A095B091D
:108F70000E9475508BA49CA4ADA4BEA4820E931E27
:108F8000A41EB51E8BA69CA6ADA6BEA64814590469
:108F90006A047B0424F44BA65CA66DA67EA66BA592
:108FA0007CA58DA59EA50E94255206EF201603E004
:108FB000300608F4AFC06093B62C7093B72C809342
:108FC000B82C9093B92C0E94ED51209147283091F4
:108FD00048282617370709F46BC160934728709318
:108FE00048288093492890934A280E9425526FA7C9
:108FF00078AB89AB9AAB8090312890903228A090C2
:109000003328B09034288BAA9CAAADAABEAA9B0193
:10901000AC0160EC71EE84E69CE40E947B51A501FA
:1090200094010E94325320E030E044EB52E40E946D
:109030007B510E94EF530E94F4516B017C0100911F
:10904000442C1091452CD8018C918E7F8C938C915F
:109050008670823009F4ABC0843009F464C0811199
:1090600069C054E0CC0CDD1CEE1CFF1C5A95D1F7F6
:1090700061C0BEE18B2E912CA12CB12C8BA69CA69D
:10908000ADA6BEA68CCFC701B6010E94ED519B01D3
:10909000AC012550310941095109A4E5B1E00E9414
:1090A000945027EF33E040E050E00E947550CA0131
:1090B000B901675E7F4F8F4F9F4F0E9425526B0112
:1090C0007C0120E030E040EF51E40E942D5318165F
:1090D0009CF420E030E044EB53E4C701B6010E9469
:1090E000765187FF10C0C701B6010E94ED516BA7F2
:1090F0007CA78DA79EA753CFC12CD12CF0EFEF2ECC
:10910000F1E4FF2EF0CFC12CD12CE4EBEE2EE3E402
:10911000FE2EE9CFAB01BC0182EB9CE20E94F31C66
:109120000E94605250CF72E0F694E794D794C794AF
:109130007A95D1F7812C912C5401A3948092522CD2
:109140009092532CA092542CB092552C9701442706
:1091500055272093462C3093472C4093482C50930E
:10916000492CC701B6018827992760934A2C709330
:109170004B2C80934C2C90934D2C2115310541059F
:109180005105A9F124013501A1E04A1A51086108ED
:109190007108613071058105910589F4C701B60137
:1091A000A30192010E94D85053014201EBCF63E02A
:1091B000CC0CDD1CEE1CFF1C6A95D1F7BBCF609375
:1091C0004A2C70934B2C80934C2C90934D2C809276
:1091D000522C9092532CA092542CB092552C209348
:1091E000462C3093472C4093482C5093492C809127
:1091F000522C9091532CA091542CB091552C019746
:10920000A109B1098093522C9093532CA093542C14
:10921000B093552C40914A2C50914B2C60914C2C82
:1092200070914D2C411551056105710561F041505A
:1092300051096109710940934A2C50934B2C60935A
:109240004C2C70934D2C4091462C5091472C6091A2
:10925000482C7091492C40934E2C50934F2C609386
:10926000502C7093512C452B462B472B21F4809189
:109270004A2C90914B2CF80184879587128613868F
:109280008081816080838091452890914628892B38
:1092900079F42BA93CA94DA95EA96FA578A989A944
:1092A0009AA90E947B510E94ED5140E00E945020FB
:1092B00080913728882309F42ACD0E94EA07609319
:1092C000BA2A7093BB2A8093BC2A9093BD2A8091BE
:1092D000B92A882309F41BCD80E00E94D22B17CD38
:1092E00050E040E061E081E00E9479216BCD50E0E8
:1092F00040E061E081E00E94DF20A5CD61E0809147
:10930000DD2C9091DE2C019709F460E083E00E944F
:10931000C72361E08091F02C9091F12C019709F422
:1093200060E081E00E94C7238091DD2C9091DE2CCB
:109330000297029738F08091F02C9091F12C0297CF
:10934000029750F58091952A9091962A8093932ABE
:109350009093942A8091DD2C9091DE2C02970297B5
:1093600040F486ED9CE20E94621A682F83E00E941E
:10937000C7238091F02C9091F12C0297029710F066
:109380000C94E24089EE9CE20E94621A682F81E010
:109390000E94C7230C94E24080914B28882309F453
:1093A00046C080915C2890915D28A0915E28B09184
:1093B0005F28892B8A2B8B2B51F40E94EA0760933C
:1093C0005C2870935D2880935E2890935F2881E0ED
:1093D000809362288091DD2C9091DE2C0297029779
:1093E00070F08091DF2C9091E02C0297029738F476
:1093F00080914B28882309F181E08093922A809103
:10940000F02C9091F12C0297029708F4A3CF809151
:10941000F22C9091F32C0297029708F09BCF809149
:109420004B28882369F081E08093912A93CF81E0D3
:109430000E94AC220E94921FCDCF0E94112BDFCF41
:109440000E94222B87CFC90165E370E00E94565528
:10945000892BC9F480915C2890915D28A0915E28A9
:10946000B0915F28892B8A2B8B2B69F00E94EA0729
:1094700020915C2830915D28621B730B6D32714026
:1094800014F00E943F238091C02A811134C1312CF5
:109490008091C12A9091C22A60E177E20E945655DC
:1094A000892BA9F480914B28882309F4A9C18091C4
:1094B000FC2C9091FD2CA091FE2CB091FF2C809360
:1094C000BA2A9093BB2AA093BC2AB093BD2A80915C
:1094D000B92A882309F4E3C08091B52A9091B62A6D
:1094E000A091B72AB091B82A4091FC2C5091FD2C44
:1094F0006091FE2C7091FF2C481B590B6A0B7B0B63
:109500004F3151056105710508F4C9C04E96A11D82
:10951000B11D8093B52A9093B62AA093B72AB09331
:10952000B82A80913728882309F4B9C06091A72A06
:109530007091A82A072E000C880B990B0E942552C7
:109540006B017C016091C52D7091C62D072E000C1A
:10955000880B990B0E9425529B01AC01C701B601F3
:109560000E947B512B013C0120911D2830911E2827
:1095700040911F28509120280E949F534B015C016D
:109580000091A52A1091A62AC090A12AD090A22AC3
:10959000E0901B28F0901C2860919F2A7091A02ACF
:1095A0006C197D09072E000C880B990B0E9425521F
:1095B000A30192010E9432532B013C01B601DD0C44
:1095C000880B990B0E9425529B01AC01C301B2018B
:1095D0000E940A510E94ED512B016091A32A7091C3
:1095E000A42A601B710B072E000C880B990B0E949C
:1095F0002552A50194010E9432534B015C01B80130
:10960000110F880B990B0E9425529B01AC01C501DB
:10961000B4010E940A510E94ED5140919D2A50913F
:109620009E2AE0919B2AF0919C2A82019B01BF0116
:109630008BEB9DE20E9404188091192890911A28C2
:109640002091A72A3091A82A280F391F2093A72AF2
:109650003093A82A4091C52D5091C62D840F951F97
:1096600082179307E4F48091992A90919A2A01969F
:109670002091972A3091982A2F5F3F4F2093972A65
:109680003093982A64E070E00E9456558093992A9E
:1096900090939A2A8091372881110E943E328091BE
:1096A000C02A10E000E0882309F4D9C0E091BE2A66
:1096B000F091BF2A628587E00E94C7238091BE2A6D
:1096C0009091BF2ADC011A962C91222311F03110BF
:1096D000BEC090E080E00E9496228091B42A811161
:1096E00004C090E080E00E94F72181E08093B42ADA
:1096F0000FEF1FEFB4C00091BE2A1091BF2A0E9445
:10970000EA072B013C01D80114968C9130E020E04F
:109710008B3218F40E9444079C0191E021303105FE
:1097200009F490E0F801928786810E9469072FEF83
:1097300033E0281B390BD80118962D933C931997C9
:109740001A963C90F80131100DC01786108A118AC4
:10975000128A8FEF9FEF838B948B85879687108675
:10976000118696CE87859089A189B289892B8A2B0B
:109770008B2B21F44786508A618A728AF801E38430
:10978000F484E586F686C8010E945224D8011B960F
:109790008D939C931C971F964D915D916D917C913B
:1097A0005297411551056105710509F470CE441AAF
:1097B000550A660A770A55962D913C915697032EC5
:1097C000000C440B550B241535054605570508F0CC
:1097D0005ECE53962D913C918217930709F457CE94
:1097E000E816F90609F053CEF8011786108A118A97
:1097F000128AE38AF48A8FEF9FEF8587968748CE97
:1098000080913728882309F462CE8091B92A81118A
:1098100063CE0E94EA070091BA2A1091BB2A2091D8
:10982000BC2A3091BD2A601B710B820B930B613EE9
:1098300073498440910508F432CF81E08093B92ABE
:1098400070E060E08BEB9DE20E947C1840CE0E94AD
:1098500052248C0181E08093B32A1092B42A809123
:10986000B22A882321F01092B32A0C94E24080910E
:10987000D12A81110C94E24080914B2881110AC0B9
:109880008091C02A811106C08091B12A882311F4E9
:109890000C94E2408091B32A8823E9F08091B02AA9
:1098A000882331F060E085E00E94C7231092B02A3F
:1098B0001092B32A81E08093AF2A8091B12A882345
:1098C00009F45BC060E080913528909136280E94B1
:1098D000F9230E943F236091472870914828809186
:1098E000492890914A2822E030E040E050E00E9470
:1098F0007550CA01B9010E9425522091312830913A
:10990000322840913328509134280E947B5120E026
:1099100030E44CE955E40E942D5308EC10E087FF39
:1099200002C008E512E08091AF2A882311F40C945C
:10993000E2400E948B07AB01BC01C801110FAA0BCA
:10994000BB0B0091AB2A1091AC2A2091AD2A30912B
:10995000AE2A800F911FA21FB31F481759076A072D
:109960007B0710F40C94E2401092AF2A70E060E0A4
:1099700080E10E9484060C94E240D090C02ADD2051
:1099800019F060E0C801A3CFE0903E28F0903F2896
:109990008091A92A9091AA2A01978093A92A90934D
:1099A000AA2A0091402810914128181619060CF493
:1099B00055C080913C2890913D288330910509F451
:1099C00079C0A8F400914028109141288130910578
:1099D000F1F0029769F100914028109141280F5F42
:1099E0001F4F0E151F05ACF110E000E032C08430AF
:1099F000910509F475C0059771F70E94914F892F61
:109A0000990F990BB7010E9456558C0127C0015040
:109A10001109C701019717FD03C00E151F050CF0B2
:109A20008C01DD24D39480179107C1F0D12C16C08E
:109A300080914228882391F10F5F1F4F17FF31C09B
:109A400081E08093422810E000E0D0904228DD20A1
:109A500029F0DD24D3940115110541F76D2DC801BE
:109A60000E94F9238091A92A9091AA2A1816190612
:109A70000CF42FCF8091DD2C9091DE2C0197029772
:109A800008F047C0000F111FF801EF5DF74D80810E
:109A900091818093A92A9093AA2A1BCF0150110982
:109AA000CDCF0E151F058CF28701015011091092C0
:109AB0004228CBCFB1E0EB16F10409F495CF8091A9
:109AC0004028909141288C010E5F1F4F0E151F05F5
:109AD0000CF4BFCF8C010095109501701127B9CF00
:109AE00080914328909144280196B7010E945655D1
:109AF0008093432890934428FC01EE0FFF1FE45B02
:109B0000F74D00811181DD24D394892B09F4A6CF70
:109B10008DCF81E090E0BDCF111195C91BCCCF93C3
:109B2000DF93DC012D91FB013191EC013883EB01D6
:109B3000288341505109CD01BF01141615068CF33D
:109B4000DF91CF910895B0E0A0E0E9EAFDE40C9444
:109B5000B1506C01D62FC72F8A017901F9010995FF
:109B6000B80197FF15C08D2F9C2FF701099597FD20
:109B700008C0B801C601F701099597FD16C0DC2D94
:109B8000CD2D8D2F9C2FCDB7DEB7E8E00C94CA50B9
:109B90008D2F9C2FF70109951816190694F3B8011B
:109BA000C601F701099597FDEACFD02FC12FE9CF64
:109BB000A8E0B0E0EEEDFDE40C94A7508C014F83DB
:109BC000588759019A013195219531092D833E839A
:109BD0006F807884600E711E6730710578F58F8113
:109BE0009885689F6001699FD00C789FD00C1124E4
:109BF000C00ED11E6C147D0420F02896E2E10C9476
:109C0000C050730113C047012F813885821A930A0F
:109C1000B701C401F50109951816190654F44F81CE
:109C20005885B401C7010E948F4D74010E151F05A0
:109C300050F3EF81F8856E0E7F1EDCCFCB01969539
:109C400087952F813885829F6001839FD00C929FDA
:109C5000D00C1124C00ED11ECB010197829F1001A0
:109C6000839F300C929F300C11247801E20CF31C7E
:109C70006730710509F442C0C701280169327105D6
:109C8000B0F183E0769567958A95E1F7629F400190
:109C9000639F900C729F900C1124C401880F991F30
:109CA00089839A83AC01400F511FB801680D791D5B
:109CB0009501C8010E94A34D2C01A601480D591D14
:109CC0009194819491089501B601C601880D991D62
:109CD0000E94A34D6C01B701680D791D9501A70184
:109CE000C701E981FA818E1B9F0B0E94A34D95014C
:109CF000AC01B601C2010E94A34D6C014F81588591
:109D0000B601C8010E948F4D4301630127011982EA
:109D10001A82EC14FD0408F446C0B801C601F5012E
:109D200009951816190654F1892B71F44F8158853D
:109D3000B601C3010E948F4D2F813885620E731EBC
:109D400081E090E089839A83EF81F885CE0EDF1E53
:109D5000E0CF892B71F44F815885B201C7010E9471
:109D60008F4D2D813E81420E531E81E090E089830C
:109D70009A83EB80FC80EC14FD04A8F0B801C701C5
:109D8000F50109952D813E812E0D3F1D2B833C83CE
:109D900097FFDFCF4F815885B701C6010E948F4DD5
:109DA000EB80FC80CDCFEF81F8852E0E3F1E200E7C
:109DB000311E29813A81232B09F58214930408F07E
:109DC0001CCF740113C06701EF81F885CE1ADF0A3A
:109DD000B701C601F50109951816190654F44F810B
:109DE0005885B601C7010E948F4D76010E151F05DB
:109DF00050F38F819885880E991EDFCF4601861813
:109E00009708A301401B510B841695060CF4A4017E
:109E10001416150634F4B601641B750BC8010E94B4
:109E20008F4D92012E193F097901A101441955095D
:109E30008F819885481B590B2417350708F4A90111
:109E40001416150634F4B101641B750BC6010E948B
:109E50008F4DEF81F885E815F90548F4C401BF017D
:109E60000E9461509501AF01C8010E94D84D2F8119
:109E700038852E153F0508F0C0CE81010E191F0947
:109E8000C701B9010E946150A3CE8F929F92AF92F9
:109E9000BF92CF92DF92EF92FF92CF93DF93EC01CC
:109EA000688179818A819B816115710581059105A0
:109EB00021F464E279ED8BE597E02DE133EF41E0A9
:109EC00050E00E94755049015A019B01AC01A7EA7C
:109ED000B1E40E9494506B017C01ACEEB4EFA5019B
:109EE00094010E94A250DC01CB018C0D9D1DAE1D82
:109EF000BF1DB7FF03C00197A109B04888839983AC
:109F0000AA83BB839F77DF91CF91FF90EF90DF9083
:109F1000CF90BF90AF909F908F9008950E94454F33
:109F2000089587E698E20E94454F0895B0E0A0E0CA
:109F30008093672890936828A0936928B0936A2833
:109F400008958F929F92AF92BF92CF92DF92EF923D
:109F5000FF92CF93DF93EC01688179818A819B81A5
:109F6000611571058105910521F464E279ED8BE5B8
:109F700097E02DE133EF41E050E00E947550490138
:109F80005A019B01AC01A7EAB1E40E9494506B0115
:109F90007C01ACEEB4EFA50194010E94A250C60E64
:109FA000D71EE81EF91EF7FE06C081E0C81AD108C8
:109FB000E10880E8F80AC882D982EA82FB82C701F8
:109FC000B6019F77DF91CF91FF90EF90DF90CF9018
:109FD000BF90AF909F908F9008958F929F92AF9275
:109FE000BF92CF92DF92EF92FF9260916B287091B7
:109FF0006C2880916D2890916E28611571058105FE
:10A00000910521F464E279ED8BE597E02DE133EFE2
:10A0100041E050E00E94755049015A019B01AC019A
:10A02000A7EAB1E40E9494506B017C01ACEEB4EF5E
:10A03000A50194010E94A250C60ED71EE81EF91E6B
:10A04000F7FE06C081E0C81AD108E10880E8F80AE6
:10A05000C0926B28D0926C28E0926D28F0926E2806
:10A06000C701B6019F77FF90EF90DF90CF90BF9030
:10A07000AF909F908F90089560936B2870936C2899
:10A0800080936D2890936E28089503D0808199273E
:10A090000895FC01E050FC4E0895262FAF93BF9326
:10A0A000E0E0F0E1328131FDFDCFDC01A050BC4E9B
:10A0B0002C932DE924BF23E020830196BF91AF911B
:10A0C0000895AA1BBB1B51E107C0AA1FBB1FA617FF
:10A0D000B70710F0A61BB70B881F991F5A95A9F751
:10A0E00080959095BC01CD010895052E97FB1EF437
:10A0F00000940E948C5057FD07D00E94D85007FC56
:10A1000003D04EF40C948C50509540953095219589
:10A110003F4F4F4F5F4F0895909580957095619593
:10A120007F4F8F4F9F4F08950E94FA50A59F900D2B
:10A13000B49F900DA49F800D911D11240895B7FF29
:10A140000C9494500E949450821B930B08952F926C
:10A150003F924F925F926F927F928F929F92AF92B7
:10A16000BF92CF92DF92EF92FF920F931F93CF9304
:10A17000DF93CDB7DEB7CA1BDB0BCDBFDEBF0994C3
:10A180002A88398848885F846E847D848C849B8487
:10A19000AA84B984C884DF80EE80FD800C811B8195
:10A1A000AA81B981CE0FD11DCDBFDEBFED010895CB
:10A1B000A1E21A2EAA1BBB1BFD010DC0AA1FBB1FCB
:10A1C000EE1FFF1FA217B307E407F50720F0A21B3D
:10A1D000B30BE40BF50B661F771F881F991F1A94AA
:10A1E00069F760957095809590959B01AC01BD01D4
:10A1F000CF010895A29FB001B39FC001A39F700D2E
:10A20000811D1124911DB29F700D811D1124911D7E
:10A2100008955058BB27AA270E9421510C94DB5265
:10A220000E94CD5238F00E94D45220F039F49F3F62
:10A2300019F426F40C94CA520EF4E095E7FB0C9442
:10A240009B52E92F0E94EC5258F3BA17620773072A
:10A250008407950720F079F4A6F50C9426530EF4A4
:10A26000E0950B2EBA2FA02D0B01B90190010C0126
:10A27000CA01A0011124FF27591B99F0593F50F43E
:10A28000503E68F11A16F040A22F232F342F442796
:10A29000585FF3CF469537952795A795F04053958E
:10A2A000C9F77EF41F16BA0B620B730B840BBAF05E
:10A2B0009150A1F0FF0FBB1F661F771F881FC2F7C9
:10A2C0000EC0BA0F621F731F841F48F487957795DD
:10A2D0006795B795F7959E3F08F0B0CF9395880F97
:10A2E00008F09927EE0F9795879508950E94775269
:10A2F00008F481E008950E948F510C94DB520E9473
:10A30000D45258F00E94CD5240F029F45F3F29F01A
:10A310000C949B5251110C9427530C94CA520E94D6
:10A32000EC5268F39923B1F3552391F3951B550B28
:10A33000BB27AA2762177307840738F09F5F5F4F18
:10A34000220F331F441FAA1FA9F335D00E2E3AF057
:10A35000E0E832D091505040E695001CCAF72BD06F
:10A36000FE2F29D0660F771F881FBB1F26173707C0
:10A370004807AB07B0E809F0BB0B802DBF01FF27F2
:10A3800093585F4F3AF09E3F510578F00C949B52E2
:10A390000C9427535F3FE4F3983ED4F3869577956A
:10A3A0006795B795F7959F5FC9F7880F911D9695AB
:10A3B000879597F90895E1E0660F771F881FBB1F07
:10A3C000621773078407BA0720F0621B730B840BB4
:10A3D000BA0BEE1F88F7E09508950E94F451689437
:10A3E000B1110C94275308950E94F45288F09F579E
:10A3F00098F0B92F9927B751B0F0E1F0660F771FA9
:10A40000881F991F1AF0BA95C9F714C0B13091F09E
:10A410000E942653B1E008950C942653672F782F9D
:10A420008827B85F39F0B93FCCF386957795679563
:10A43000B395D9F73EF490958095709561957F4FCF
:10A440008F4F9F4F0895E89409C097FB3EF4909575
:10A450008095709561957F4F8F4F9F4F9923A9F0FD
:10A46000F92F96E9BB279395F6958795779567958C
:10A47000B795F111F8CFFAF4BB0F11F460FF1BC0D0
:10A480006F5F7F4F8F4F9F4F16C0882311F096E963
:10A4900011C0772321F09EE8872F762F05C0662311
:10A4A00071F096E8862F70E060E02AF09A95660FCA
:10A4B000771F881FDAF7880F9695879597F9089583
:10A4C0000E940E5390F09F3748F4911116F00C94AF
:10A4D000275360E070E080E89FEB089526F41B1698
:10A4E000611D711D811D0C94A1520C94BC52990FD9
:10A4F0000008550FAA0BE0E8FEEF16161706E8074E
:10A50000F907C0F012161306E407F50798F0621B6E
:10A51000730B840B950B39F40A2661F0232B242B43
:10A52000252B21F408950A2609F4A140A6958FEF62
:10A53000811D811D089597F99F6780E870E060E0B4
:10A540000895882371F4772321F09850872B762F74
:10A5500007C0662311F499270DC09051862B70E037
:10A5600060E02AF09A95660F771F881FDAF7880F48
:10A570009695879597F908959F3F31F0915020F473
:10A58000879577956795B795880F911D96958795CF
:10A5900097F908959FEF80EC089500240A94161609
:10A5A000170618060906089500240A9412161306C1
:10A5B000140605060895092E0394000C11F488234F
:10A5C00052F0BB0F40F4BF2B11F460FF04C06F5F6B
:10A5D0007F4F8F4F9F4F089557FD9058440F551F41
:10A5E00059F05F3F71F04795880F97FB991F61F015
:10A5F0009F3F79F087950895121613061406551F8C
:10A60000F2CF4695F1DF08C0161617061806991FF7
:10A61000F1CF869571056105089408950E94F45262
:10A62000A0F0BEE7B91788F4BB279F3860F4161670
:10A63000B11D672F782F8827985FF7CF869577957C
:10A640006795B11D93959639C8F30895E894BB2793
:10A6500066277727CB0197F908950E94775208F46F
:10A660008FEF08950E9445530C94DB520E94CD5207
:10A6700038F00E94D45220F0952311F00C949B5294
:10A680000C94CA5211240C9427530E94EC5270F37C
:10A69000959FC1F3950F50E0551F629FF001729F87
:10A6A000BB27F00DB11D639FAA27F00DB11DAA1F96
:10A6B000649F6627B00DA11D661F829F2227B00DE3
:10A6C000A11D621F739FB00DA11D621F839FA00D6E
:10A6D000611D221F749F3327A00D611D231F849FBE
:10A6E000600D211D822F762F6A2F11249F57504015
:10A6F0009AF0F1F088234AF0EE0FFF1FBB1F661F90
:10A70000771F881F91505040A9F79E3F510580F058
:10A710000C949B520C9427535F3FE4F3983ED4F380
:10A72000869577956795B795F795E7959F5FC1F7FC
:10A73000FE2B880F911D9695879597F90895FA013C
:10A74000EE0FFF1F309621053105A1F1611571054E
:10A7500061F48038BFE39B0749F168949038810524
:10A7600061F08038BFEF9B0741F099234AF5FF3F26
:10A77000E1053105210519F1E8940894E795D9011F
:10A78000AA2329F4AB2FBE2FF85FD0F310C0FF5FD0
:10A7900070F4A695E0F7F73950F019F0FF3A38F465
:10A7A0009F779F930DD00F9007FC9058089546F027
:10A7B0000C94CA5260E070E080E89FE308954FE790
:10A7C0009F775F934F933F932F930E94BE542F9197
:10A7D0003F914F915F910E9432530C941B540E9401
:10A7E000F452E8F09E37E8F09639B8F49E3848F411
:10A7F000672F782F8827985FF9CF8695779567958B
:10A8000093959539D0F3B62FB1706B0F711D811DE3
:10A8100020F487957795679593950C94A1520C94A5
:10A82000BC520C94275329F416F00C949B520C94B0
:10A8300026530C94CA520E94F452A8F39638A0F7FB
:10A8400007F80F92E8942BE33AEA48EB5FE70E949F
:10A8500048530F920F920F924DB75EB70F920E941E
:10A860000655E0EAF0E00E944D544F915F91EF9160
:10A87000FF91E595EE1FFF1F49F0FE57E068442762
:10A88000EE0F441FFA95E1F74195550B0E94805455
:10A890000F9007FE0C9474540895DF93CF931F9389
:10A8A0000F93FF92EF92DF927B018C01689406C0B8
:10A8B000DA2EEF010E944553FE01E894A5912591FF
:10A8C000359145915591A6F3EF010E942151FE016A
:10A8D0009701A801DA9469F7DF90EF90FF900F914C
:10A8E0001F91CF91DF9108959B01AC0160E070E072
:10A8F00080E89FE30C947B510C949B520C94BC52C7
:10A900000E94F452D8F39923C9F3940F511DA3F375
:10A910009150504094F059F0882332F0660F771F21
:10A92000881F91505040C1F79E3F51052CF7880F6A
:10A93000911D9695879597F908955F3FACF0983EE5
:10A940009CF0BB27869577956795B79508F4B1601D
:10A950009395C1F7BB0F58F711F460FFE8CF6F5F15
:10A960007F4F8F4F9F4FE3CF0C94275316F00C94DB
:10A97000BC520C94CA5268940C949B520E94F4529C
:10A98000A8F39923C1F3AEF3DF93CF931F930F93F3
:10A99000FF92C92FDD2788232AF02197660F771FA2
:10A9A000881FDAF720E030E040E85FEB9FE388396A
:10A9B00020F0803E38F021968F770E940A51E8EC13
:10A9C000F0E004C00E940A51E5EFF0E00E944D540F
:10A9D0008B01BE01EC01FB2E6F5771097595771F36
:10A9E000880B990B0E94255228E132E741E35FE38F
:10A9F0000E944553AF2D9801AE01FF900F911F911A
:10AA0000CF91DF910E9421510C94DB52FA01DC01BD
:10AA1000AA0FBB1F9B01AC01BF5728F42227332785
:10AA20004427507820C0B75190F4AB2F00244695AE
:10AA300037952795011CA395D2F3002071F0220FC2
:10AA4000331F441FB395DAF30ED00C9409516130D3
:10AA50007105A0E88A07B94630F49B01AC0166276E
:10AA6000772788279078309621F02083318342839E
:10AA700053830895DB018F939F930E949450BF915D
:10AA8000AF91A29F800D911DA39F900DB29F900D3D
:10AA900011240895991B79E004C0991F961708F0B6
:10AAA000961B881F7A95C9F78095089597FB072E06
:10AAB00016F4009407D077FD09D00E94615007FC7E
:10AAC00005D03EF4909581959F4F089570956195BE
:10AAD0007F4F0895EE0FFF1F0590F491E02D09942C
:10AAE0000E94FA50332312F48A1B9B0B0C947A5564
:10AAF0000E94FA50B7FF0895821B930B089597FDAB
:10AB00001094002E083098F00850232F342F452F32
:10AB1000562F672F782F892F912DF4CF1594979565
:10AB200087957795679557954795379527950A9512
:10AB3000AAF71124002D08950024A7FD00942A17D8
:10AB400030054005500560057005800590050895A5
:10AB50000F931F93CF93DF938230910510F482E01F
:10AB600090E0E091092EF0910A2E30E020E0B0E074
:10AB7000A0E0309799F42115310509F44AC0281B4B
:10AB8000390B24303105D8F58A819B816115710517
:10AB900089F1FB0182839383FE0111C040815181C1
:10ABA0000281138148175907E0F04817590799F4B3
:10ABB000109761F012960C93129713961C9332968D
:10ABC000CF01DF91CF911F910F9108950093092E2E
:10ABD00010930A2EF4CF2115310551F04217530777
:10ABE00038F0A901DB019A01BD01DF01F801C1CFF5
:10ABF000EF01F9CF8093092E90930A2ECDCFFE015D
:10AC0000E20FF31F819391932250310928833983F6
:10AC1000D7CF2091072E3091082E232B41F420917D
:10AC20007128309172282093072E3093082E20919E
:10AC30006F28309170282115310541F42DB73EB7AA
:10AC40004091732850917428241B350BE091072EF6
:10AC5000F091082EE217F307A0F42E1B3F0B2817E4
:10AC6000390778F0AC014E5F5F4F2417350748F085
:10AC70004E0F5F1F4093072E5093082E81939193A0
:10AC80009FCFF0E0E0E09CCFCF93DF930097E9F017
:10AC9000FC01329712821382A091092EB0910A2EE4
:10ACA000ED0130E020E01097A1F420813181820F86
:10ACB000931F2091072E3091082E2817390709F08D
:10ACC00061C0E093072EF093082EDF91CF91089595
:10ACD000EA01CE17DF07E8F54A815B819E01411545
:10ACE0005105B1F7E901EA83FB8349915991C40FFA
:10ACF000D51FEC17FD0761F4808191810296840FC6
:10AD0000951FE90188839983828193818A839B833C
:10AD1000F0E0E0E012968D919C9113970097B9F5C1
:10AD20002D913C911197CD010296820F931F209196
:10AD3000072E3091082E2817390739F6309751F52C
:10AD40001092092E10920A2EA093072EB093082E6F
:10AD5000BCCFC283D38340815181840F951FC81714
:10AD6000D90761F44E5F5F4F88819981480F591F61
:10AD7000408351838A819B8182839383211531058E
:10AD800009F0B0CFE093092EF0930A2E9ECFFD017B
:10AD9000DC01C0CF12821382D7CF81E090E0F8941B
:08ADA0000C94D256F894FFCF89
:10ADA8000100010001000100010001000100010093
:10ADB80083F086F08AF08FF093F00BF1A2F0A5F003
:10ADC800A8F0ABF0AEF0F5EF97F099F09BF09EF09D
:10ADD800A1F0A4F0A7F0AAF0ADF0000000008001F7
:10ADE80000000003000080030000000400001E00B3
:10ADF80000007A00000072010000E80300008813D8
:10AE080000000000FFFF0100FFFF02000300FFFF3A
:10AE18000400FFFF05000600070018000C000600EC
:10AE28000100FFFF0200FFFF03000400FFFF050011
:10AE3800FFFF060007000800030201000C0D0405CF
:10AE480000000003000102000001010000000000F2
:10AE58000000000000000000000000000000B6092B
:10AE6800B20900093D90D00380841E90D00324F4D9
:10AE7800000024F440420F00127A40420F90D003A1
:10AE8800000000000000803F0000A040C2F0C9F0B0
:10AE9800D1F0D8F0E1F0E9F0F0F0F8F002F10DF1BE
:10AEA8000504000506020401030001000102030273
:10AEB80001000203040502030504000000001C054C
:10AEC8008F0581046D05B2049004A404591ACC06B8
:10AED800BE041A0600000000C4095928140AE5092E
:10AEE800C509180BC70AE8291E0A680B620BA728B0
:10AEF8005A0B00000000E60CC10C2A1A970CBA0C79
:10AF0800A70C980CB70D720D650D610D280D090D74
:10AF1800010D370D2F0D700C6B0C20100120400413
:10AF280010020801020102040804020104081020AA
:10AF380004082010020200050201050004010104B2
:10AF480004040303030305050303000001010000D3
:10AF58000000D3168F052A1A291AEC1090144D14E4
:10AF6800E4136313A4137F197F146B10CF1081129D
:10AF7800F21270127C180418A517FD28610F000042
:10AF880000004D1A451A3D1A351A2D1A6F666600CB
:10AF98005365742000536574207377696E672000C9
:10AFA8002D002A002B00202000202030004D69634E
:10AFB800726F74696D696E6773004D756C7469732F
:10AFC80074657073005B005D00536574207374656D
:10AFD80070733A00537465702031207365740044AF
:10AFE80046414D205468696E670076312E3700431C
:10AFF8006F6E66696775726174696F6E005363720C
:10B0080065656E73617665723A00436F6C6F757231
:10B018003A00416C6C6F7720666173743A00496E30
:10B0280076657274204C43443A005050514E3A00B1
:10B038004D4944492063683A0043616C6962726112
:10B04800746500506C6179204332004F4B20280012
:10B058002900506C6179204334004F4B00446F6ED7
:10B0680065004661696C6564005365742073746596
:10B0780070733A200042504D3A20004F6E004F66E0
:10B088006600426C75650052656400416C6C00385E
:10B0980000390031300031310031320031330031B4
:10B0A8003400313500313600496E742E004578740D
:10B0B8002E004D494449003234004E6F726D616C68
:10B0C800005265766572736500426F756E63650040
:10B0D8004F64642F4576656E0053687566666C65C7
:10B0E8000052616E646F6D004356204D6F646500B9
:10B0F8004D494449204D6F6465005365742073744D
:0BB1080065702031005377696E67000E
:10B113001027FFFFFFFF3C028B0118BFF0A1F0AE29
:10B12300F00024F400015A00010200FFFF00008038
:10B133003F010001000100010001000100010001C5
:10B14300000000803FFFFF010000484300000800AB
:10B153000000010000000078000000000000010072
:10B1630002000300040005000600070000000000C1
:10B17300000000FFFFFFFF010000000100000000CE
:06B18300000B2E8000000D
:00000001FF
